:100000000C94A9020C94C6020C94C6020C94C6026D
:100010000C94C6020C94C6020C94C6020C94C60240
:100020000C94C6020C94C6020C94C6020C94C60230
:100030000C94C6020C94C6020C94C6020C94C60220
:100040000C940C2D0C94C6020C94C6020C94C6029F
:100050000C94C6020C94C6020C94C6020C94C60200
:100060000C94C6020C94C602312E30322E30300071
:100070004845414400474554202F0054532D4E54C9
:1000800050434B30315F58585858006E74702E6A88
:1000900073742E6D666565642E61642E6A70006EE1
:1000A00074702E6E6963742E6A70008B009F00213D
:1000B0000441043031323334353637383941424324
:1000C00044454600485454502F312E3120323030B0
:1000D00020485454500D0A436F6E6E656374696F07
:1000E0006E3A20636C6F73650D0A436F6E74656EB4
:1000F000742D547970653A20746578742F68746D26
:100100006C0D0A43616368652D436F6E74726F6C8A
:100110003A206E6F2D63616368650D0A436F6E74DC
:10012000656E742D4C616E67756167653A20656E0A
:100130000D0A0D0A00485454502F312E3120323010
:1001400030204F4B0D0A436F6E6E656374696F6E9E
:100150003A20636C6F73650D0A436F6E74656E743D
:100160002D547970653A20746578742F68746D6CBD
:100170000D0A43616368652D436F6E74726F6C3A4C
:10018000206E6F2D63616368650D0A436F6E746541
:100190006E742D4C616E67756167653A20656E0DF2
:1001A0000A0D0A3C21444F43545950452048544DB0
:1001B0004C205055424C494320222D2F2F5733437A
:1001C0002F2F4454442048544D4C20342E3031209D
:1001D0005472616E736974696F6E616C2F2F454E36
:1001E000222022687474703A2F2F7777772E773316
:1001F0002E6F72672F54522F68746D6C342F6C6F92
:100200006F73652E647464223E3C48544D4C3E3CF2
:10021000484541443E3C5449544C453E54532D4E70
:1002200054502D434C4F434B2053455455503C2F75
:100230005449544C453E3C2F484541443E3C424F76
:100240004459204247434F4C4F523D222346464695
:100250004646464646223E3C43454E5445523E3C69
:10026000423E00223E3C2F464F524D3E3C42523EC3
:100270003C464F4E5420434F4C4F523D224752452F
:10028000454E223E56414C55452053415645443C2F
:100290002F464F4E543E3C42523E00223E3C42527C
:1002A0003E3C42523E3C494E5055542054595045D4
:1002B0003D225355424D4954222056414C55453D0F
:1002C000224150504C59223E3C2F464F524D3E0049
:1002D0004E31004E3200D002D302534552564552A1
:1002E00031005345525645523200DA02E2024000D4
:1002F00060006E732E6367690066617669636F00E4
:10030000F202F90254494D452053455256455220B8
:1003100053455454494E470020485454502F003CF4
:1003200042523E3C2F43454E5445523E3C2F424F95
:1003300044593E3C2F48544D4C3E0022204D4554DC
:10034000484F443D22474554003C2F423E3C4252D8
:100350003E3C464F524D20414354494F4E3D2200B2
:10036000222056414C55453D220022204D41584CFB
:10037000454E4754483D2200222053495A453D22CC
:10038000003C42523E3C494E505554205459504531
:100390003D225445585422204E414D453D220022D5
:1003A0003E3C42523E0054494D4552204F46460085
:1003B00053494E474C45204D4F444500434F4E5402
:1003C000494E5545204D4F444500A603B003BC039C
:1003D0000209000509000509534D545754465300BE
:1003E0002D2D2054494D4552204D4F4445202D2D53
:1003F000004F464654494D45004F4E54494D450027
:1004000020203A20203A2020004F464620574441E1
:10041000593A004F4E2020574441593A0053554E07
:10042000004D4F4E00545545005745440054485523
:100430000046524900534154004149555454532DEC
:100440004E54502D434C4F434B303100454E4332B8
:10045000384A3630205245563A00494E49544941AF
:100460004C495A494E472E2E2E00494E4954494177
:100470004C495A4544004B4559494E505554204922
:100480004C4C4547414C0043414C2052454D3A00AD
:100490003D044C045A046A0476048704566572735A
:1004A000696F6E00504C4541534520434845434BCE
:1004B000204B455900504C4541534520524553452A
:1004C00054004D41433A0044484350434E543A008F
:1004D00054494D45523A009C04A404B504C204C7D3
:1004E00004D004455850495245442000205245420A
:1004F000494E44200052454E4557414C2000494E3C
:1005000046494E49545900E304EC04F504FE042D19
:100510002D2F2D2D202D2D3A2D2D3A2D2D004F46EE
:10052000460053474C00434E54001E052205260545
:10053000C0F9A4B0999282F88090FF88FBC1872A05
:100540002A3A2A2A3A2A2A002D2D3A2D2D3A2D2DE3
:10055000000011241FBECFEFD8E0DEBFCDBF12E0F8
:10056000A0E0B1E0E6E7FCE702C005900D92AA36F4
:10057000B107D9F715E0AAE6B2E001C01D92A43E8A
:10058000B107E1F70E9404050C94393E0C94000079
:100590006091B905262F30E08091230190912401CC
:1005A00028173907C9F55091BA05252F30E08091F9
:1005B0002101909122012817390771F54091BB055F
:1005C000242F30E080911F019091200128173907D6
:1005D00019F55F9A8091B5058130F1F48091BD05E0
:1005E0006817A1F48091BE05581781F48091BF056A
:1005F000481761F41092B50501C0A895F999FDCF8F
:1006000085E390E060E00E94F63D089581E090E08F
:100610009093B7058093B60508958091BD0590E04D
:1006200020912301309124018217930721F58091B5
:10063000BE0590E02091210130912201821793079D
:10064000D1F48091BF0590E020911F0130912001ED
:100650008217930781F45F988091B505813059F432
:100660001092B50501C0A895F999FDCF85E390E0FA
:1006700060E00E94F63D0895A0E2B0E0E2E4F3E01D
:100680000C94FD3C0E94D70C82E00E94ED3201C028
:10069000A895F999FDCF8EE090E060E570E00E94AA
:1006A000343E01C0A895F999FDCF8CE090E06AE056
:1006B00070E00E94343E01C0A895F999FDCF85E312
:1006C00090E060E00E941E3E01C0A895F999FDCF20
:1006D00086E390E040E050E060E070E00E942C3E55
:1006E00001C0A895F999FDCF8AE390E040E050E081
:1006F00060E070E00E942C3E01C0A895F999FDCF02
:100700008E010F5F1F4FC8016BE870E00E944B3DE8
:10071000C80160E470E040E250E00E94143E01C075
:10072000A895F999FDCF8E010F5F1F4FC8016FE9A2
:1007300070E00E944B3DC80160E670E040E250E08E
:100740000E94143E01C0A895F999FDCF80EC90E07D
:1007500068E572E00E94343E01C0A895F999FDCF8A
:1007600082EC90E06CED75E00E94343E01C0A895EB
:10077000F999FDCF8EE390E065EA73EC0E94343E78
:10078000A096E4E00C94193DA4E0B0E0EAECF3E0BC
:100790000C94FD3C8E010F5F1F4FC80160E00E946A
:1007A00088228130B1F489819A81AB81BC81009724
:1007B000A105B10571F4C80161E00E948822813071
:1007C00041F489819A81AB81BC810097A105B10573
:1007D00039F081E090E090930A018093090104C010
:1007E00010920A01109209012496E4E00C94193D3C
:1007F0000E94730E89B180958770873069F40E94DA
:100800003C030E94D70C83E00E94ED3282E00E94FC
:10081000E032A895FECFA895F999FDCF8EE390E040
:100820000E94E03D855A934C21F00E943C0301C098
:10083000A895F999FDCF8EE090E00E94E03D90935D
:1008400014038093130301978E5F9F4F40F080E560
:1008500090E0909314038093130301C0A895F99935
:10086000FDCF8CE090E00E94E03D9C013F7730930B
:10087000BC042093BB0401978E5F9F4F30F08CE344
:1008800090E09093BC048093BB048091AB05909161
:10089000AC05019711F084E101C085E18093BE04AD
:1008A00083E995E06BE770E00E944B3D8091040185
:1008B0006EE975E00E940E2B8091050160EA75E0FB
:1008C0000E940E2B01C0A895F999FDCF85E390E019
:1008D0000E94D23D8093B50501C0A895F999FDCF3E
:1008E00086E390E00E94DA3D6093B8057093B90505
:1008F0008093BA059093BB0501C0A895F999FDCFE7
:100900008AE390E00E94DA3D6093BC057093BD05D8
:100910008093BE059093BF0580E490E061E274E0AF
:100920004BE850E00E94050E80E690E061E474E040
:100930004FE950E00E94050E0E94C40301C0A89533
:10094000F999FDCF80EC90E00E94E03D9093820405
:100950008093810401978E5F9F4F40F088E592E07D
:10096000909382048093810401C0A895F999FDCFEA
:1009700082EC90E00E94E03D909386048093850491
:100980008F5F9F4F31F48CED95E0909386048093B8
:1009900085041092AF050895EF92FF920F931F9375
:1009A000E0908304F09084040027F7FC0095102F5A
:1009B00083E491E06FE171E00E94BD2CE61AF70A32
:1009C000080B190BB701C8011F910F91FF90EF9011
:1009D00008950F931F938C010E94AF2B005110407C
:1009E0006F717070600F711F709384046093830443
:1009F000A3E4B1E0EFE1F1E082E101900D928150DA
:100A0000E1F71F910F910895A4E0B0E0EAE0F5E06E
:100A10000C94F23CF8948BEC8093640080E880BFE7
:100A200014E015B918B880E68BB98FE284B98FE36A
:100A300087B980EF8AB988E090E00E94DA3D609340
:100A40008704709388048093890490938A0480E1DA
:100A50008CBD16BC14BC15BD81E080936E0084B7BC
:100A6000992787FD909580FD0CC081FD04C082FD13
:100A700002C083FF06C081E090E09093AC058093B4
:100A8000AB0514BE2CE088E190E00FB6F894A89571
:100A9000809360000FBE20936000789410E51CBD29
:100AA0000E94173280E18CBD0E94300D0E94F80335
:100AB0001CBD299A89E190E00E94700D0E94E8080F
:100AC000882331F484E162EA7AE00E941708FFCFBC
:100AD0000E94500B8EE190E00E947F0D80E00E940A
:100AE000ED3280E00E94E03288E061E048E650E0CC
:100AF0000E94080D8EEE92E00E947F0D0E94D70C9E
:100B00008091BE048823D1F081E090E09093C004EE
:100B10008093BF04ABE0B1E0EFE1F1E082E101904E
:100B20000D928150E1F78091BE04843119F40E9446
:100B3000DD1808C086E10E94BB1904C01092C004F1
:100B40001092BF041092AC051092AB050E94770D75
:100B50005C013E010894611C711C41E0842E912CC3
:100B600001E030EC532EA8950E94DD12823019F47A
:100B70000E94591109C0833019F40E94BC1704C0A7
:100B8000843009F50E942915182F0E94710911233C
:100B9000D1F0163091F48091B0058823A1F0A3E440
:100BA000B1E0EFE1F1E082E101900D928150E1F7D7
:100BB000109290051092B00506C01B3121F480E41C
:100BC00090E00E94E904F8948091C6059091C705D1
:100BD0009093AE058093AD051092C7051092C6059F
:100BE00078948091AD059091AE05019709F0B5C05C
:100BF000F8948091C2059091C305A091C405B0916D
:100C0000C50589839A83AB83BC837894C3010E9412
:100C1000F30E009729F450920701009306010EC0CD
:100C2000A1E3B1E0FC0182E101900D928150E1F776
:100C300081E391E06FE171E00E94DA2C0E944C0F99
:100C40000E94E2200E94BE1A8091090190910A013F
:100C5000019721F0CC24DD24760137C08091B005C6
:100C6000882321F0CC24DD24760117C00E94CC0417
:100C70006B017C01161617061806190674F0809190
:100C8000DA029091DB02A091DC02B091DD020097C4
:100C9000A105B10511F00093B005809107018034E2
:100CA000A1F48091350190913601892B71F48091E6
:100CB000330190913401892B41F48091310190915D
:100CC0003201892B11F40093B0058091B50588237A
:100CD00011F1813059F48091B6059091B7050197D3
:100CE00011F40E940D030E94C80215C0C4010090B7
:100CF0002B0102C0880F991F0A94E2F7182F8091E8
:100D0000B805812311F00E94C8028091BC05182308
:100D100011F00E940D038FE191E00E942332809137
:100D2000A705882319F40E94B83317C08430A9F4AA
:100D30008091090190910A01892B21F08091B005E1
:100D4000882321F080E00E94D93205C080E0B701FD
:100D5000A6010E942E330E9478338091A805882333
:100D600011F18130E1F48091830490918404803406
:100D7000910514F480E490E0880F991F24E08130FD
:100D8000920714F080E094E00E94E904A3E4B1E04B
:100D9000EFE1F1E082E101900D928150E1F71092D4
:100DA000B00510920601809190058823B9F00E9449
:100DB00033218823C9F080518B3058F4A3E4B1E08B
:100DC000EFE1F1E082E101900D928150E1F70E94A4
:100DD000A522109290051092B00506C010928F05C2
:100DE00010929205109291050E942F23882341F0C2
:100DF000109290051092B00580E490E00E94E90402
:100E00008091AD059091AE050197F1F48091EF02CC
:100E1000882359F080910003815080930003882338
:100E200021F480E090E00E94EE1480910103882379
:100E300059F080911203815080931203882321F48A
:100E400081E090E00E94EE148091A9059091AA059E
:100E5000019711F40E9453341092AA051092A9052B
:100E60001092AE051092AD051092A8050E94770D64
:100E70008A199B09059740F10E94770D5C010E9439
:100E8000940D0E94A30D8823F9F01091A7058131DC
:100E900021F41F5F153098F413C0833119F40E94B8
:100EA0007F300DC0843119F40E94300D09C08531A6
:100EB00011F45F9A09C0863139F45F9805C010E0DB
:100EC0001093A7050E94533480910601882331F4C2
:100ED0009092B2058092B1055D9805C01092B2055E
:100EE0001092B1055D9A8091DA029091DB02A09197
:100EF000DC02B091DD020097A105B10531F00E943E
:100F00002909813011F45E982ECE5E9A2CCE8EBDCA
:100F10000DB407FEFDCF08952A988EBD0DB407FECF
:100F2000FDCF1EBC0DB407FEFDCF8EB52A9A0895E5
:100F30002A988EBD0DB407FEFDCF1EBC0DB407FE72
:100F4000FDCF8EB51EBC0DB407FEFDCF8EB52A9A1F
:100F500008952A98805C8EBD0DB407FEFDCF6EBD4E
:100F60000DB407FEFDCF2A9A08950F931F93182FF3
:100F70000E949807082F812F8F5F0E949807982F53
:100F8000802F1F910F9108950F931F93182F072FF4
:100F90000E94A907812F8F5F602F0E94A9071F91D0
:100FA0000F9108952A9880588EBD0DB407FEFDCF8D
:100FB0006EBD0DB407FEFDCF2A9A08952A9880567B
:100FC0008EBD0DB407FEFDCF6EBD0DB407FEFDCF87
:100FD0002A9A08951F93182F8FE163E00E94DE077D
:100FE0008FE1612F0E94D2071F9108951F93182F40
:100FF00082E00E94EA0784E1612F0E94A90782E152
:1010000061E00E94A90783E00E94EA078AE00E944B
:10101000980780FDFBCF82E00E94EA0782E160E052
:101020000E94A90788E10E94B5071F910895FF92C9
:101030000F931F93F82E8B0182E00E94EA0784E150
:101040006F2D0E94A90786E1B8010E94C40783E0C2
:101050000E94EA078AE00E94980780FDFBCF1F915B
:101060000F91FF9008952A988AE38EBD0DB407FE74
:10107000FDCF1EBC0DB407FEFDCF8EB52A9A089594
:101080002A988AE38EBD0DB407FEFDCF1EBC0DB4B9
:1010900007FEFDCF9EB51EBC0DB407FEFDCF8EB57D
:1010A0002A9A08952A988AE38EBD0DB407FEFDCFD3
:1010B0001EBC0DB407FEFDCF9EB51EBC0DB407FED1
:1010C000FDCF8EB51EBC0DB407FEFDCF7EB51EBC98
:1010D0000DB407FEFDCF6EB52A9A0895FC012A983B
:1010E0008AE38EBD0DB407FEFDCF20E030E008C0DE
:1010F0001EBC0DB407FEFDCF8EB581932F5F3F4F11
:1011000026173707A8F32A9A0895982F2A988AE76E
:101110008EBD0DB407FEFDCF9EBD0DB407FEFDCF05
:101120002A9A0895282F2A988AE78EBD0DB407FEC3
:10113000FDCF9EBD0DB407FEFDCF2EBD0DB407FE45
:10114000FDCF2A9A0895282F2A988AE78EBD0DB4DC
:1011500007FEFDCF9EBD0DB407FEFDCF2EBD0DB425
:1011600007FEFDCF7EBD0DB407FEFDCF6EBD0DB4F5
:1011700007FEFDCF2A9A0895FC012A988AE78EBDC2
:101180000DB407FEFDCF20E030E008C080818EBDA9
:101190000DB407FEFDCF2F5F3F4F3196261737075F
:1011A000A8F32A9ACB010895282F2A988AE78EBDA2
:1011B0000DB407FEFDCF80E090E005C02EBD0DB45C
:1011C00007FEFDCF019686179707C0F32A9A089568
:1011D0000F931F938FE160E00E94A90780E160E018
:1011E00070E00E94C40782E16FEF7FE10E94C407B4
:1011F0008AE06FEF7FE10E94C40783E00E94EA0764
:1012000087E067E00E94A90787E00E948C0780FDC5
:10121000FBCF87E062E00E94DE078FE160E30E947F
:10122000D2078FE10E948C0785FDFBCF80E00E94F2
:10123000EA0786E10E948C07082F87E10E948C074D
:10124000182F80E00750184F09F481E01F910F918B
:10125000089581E00E94F607969587959695879563
:1012600081700895EF92FF920F931F938C0180E09D
:101270000E94EA0780E00E94B507F82EE92E6091EF
:101280007802709179026A5F7F4F600F711F89E168
:10129000683D780710F0685D794180E00E94C407DE
:1012A0008F2D9E2D1F910F91FF90EF900895EF923B
:1012B000FF920F931F938C0180E00E94EA0782E067
:1012C0000E94B507F82EE92E0752164E82E0B801AB
:1012D0000E94C4078F2D9E2D1F910F91FF90EF90BC
:1012E00008950F931F9300917A0210917B02015091
:1012F000104080E00E94EA078EE160E40E94D2077D
:10130000B80189E1083D180710F067ED79E18CE03C
:101310000E94C4071F910F910895A7E0B0E0E3E990
:10132000F9E00C94F73C8C01E0907D02F0907E0295
:10133000E80EF91E82E0B8010E94C40780E00E9416
:10134000850884E0B8010E94C40786E0B7010E94C6
:10135000C4078FE160E80E94D2078FE160E80E9435
:10136000DE078CE16AE00E94DE078FE168E00E9400
:10137000D20780917C028550823008F068C000E07E
:1013800010E08CE10E948C078A7031F40F5F1F4FD0
:1013900083E0083E1807A9F78CE10E948C0781FDC5
:1013A00005C083E0083E180708F451C08FE168E0EB
:1013B0000E94DE0780E00E94B5075C0186E00E9483
:1013C000B5076C010894C11CD11C80E0B6010E94D5
:1013D000C4078E010F5F1F4FC80167E070E00E94D5
:1013E0006E08EE24F02E012F8CE10E948C0781FF05
:1013F0002AC08C8185FF27C08FE160E80E94D20758
:101400008FE160E80E94DE078CE16AE00E94DE075F
:101410008FE168E00E94D2078CE10E948C078A70FD
:10142000D9F38FE168E00E94DE0780E0B6010E94F8
:10143000C4078F2D902F67E070E00E946E08E39440
:1014400080E1E81689F680E0B5010E94C40727967E
:10145000EAE00C94133DA0E0B0E0E1E3FAE00C9484
:10146000F83CB82E282F392F6901EE24FF2487017C
:1014700011C00E943308D82F0E943308C82FCE0114
:10148000A0E0B0E0E80EF91E0A1F1B1F8EEF9FEFD1
:10149000C80ED91E92E0C916D10458F7C701D80169
:1014A0009C01AD01B0FE0BC00E943308D82FC0E0F4
:1014B0009E0140E050E02E0D3F1D401F511F203087
:1014C00080E0380781E0480780E05807A0F0CA01B3
:1014D00040E050E0A0E0B0E0280F391F4A1F5B1F3A
:1014E000203090E0390791E0490790E0590718F063
:1014F000C90101969C01C901CDB7DEB7E9E00C94A2
:10150000143D0F931F938B010E943209C8010E9462
:101510002B0A9C0120953095C9011F910F910895C8
:10152000EF92FF920F931F938C017B0180E00E944A
:10153000EA070752164E80E0B8010E94C407C701AF
:101540000E942B0A9C0120953095C9011F910F9193
:10155000FF90EF900895A0E0B0E0E1EBFAE00C948A
:10156000F93C6C017B018A014115510509F444C025
:101570004130510551F40E943209C7010E945709B8
:101580000E9433080E94850837C080E00E94EA0765
:10159000C0917802D09179022696CC0DDD1D89E1AB
:1015A000C83DD80710F0C85DD94180E1BE010E9456
:1015B000C407B801615070406C0F7D1F99E1683D10
:1015C000790710F0685D794182E10E94C40789EDD6
:1015D00099E1E80EF91E84E1B7010E94C4078FE18A
:1015E00060E10E94DE078FE160E20E94D2078FE196
:1015F0000E948C0785FDFBCFCDB7DEB7E8E00C94E9
:10160000153DFC012A988AE38EBD0DB407FEFDCF7F
:1016100020E030E00AC01EBC0DB407FEFDCF8EB541
:1016200081932F5F3F4F841719F02617370798F3E0
:1016300010822A9AC90108950F931F93CF93DF93C5
:101640008C01C0E0D0E003C00E9433082196C0178F
:10165000D107D0F3DF91CF911F910F910895CF93D0
:10166000DF93EC010E94523DAC012A988AE78EBDBF
:101670000DB407FEFDCF20E030E00AC0FE01E20F0E
:10168000F31FE491EEBD0DB407FEFDCF2F5F3F4F7A
:101690002417350798F32A9ACA01DF91CF9108954C
:1016A0001F938EE160E20E94DE0789E190E00E94D4
:1016B000700D299889E190E00E94700D299A89E1C6
:1016C00090E00E94700D1FEF2A981EBD0DB407FE1A
:1016D000FDCF2A9A89E190E00E94700D8DE10E9471
:1016E0008C0783FDF1CF80FFEFCF8FE160EC0E948C
:1016F000A9078EE160E80E94A90788E060E070E039
:101700000E94C4078CE067ED79E10E94C4078AE07B
:1017100067ED79E10E94C40784E068ED79E10E94F9
:10172000C40781E00E94EA0788E161EA0E94A907F4
:1017300082E00E94EA0780E06DE00E94A90781E054
:1017400060E00E94A90782E062E30E94A9078AE0A4
:101750006EEE75E00E94C40786E062E17CE00E94C4
:10176000C40784E062E10E94A90783E060E40E946C
:10177000A90789E06FE30E94A90783E00E94EA07B6
:1017800085E160E00E94A90784E0609100010E9469
:10179000A90785E0609101010E94A90782E060919C
:1017A00002010E94A90783E0609103010E94A9073A
:1017B00080E0609104010E94A90781E06091050129
:1017C0000E94A90782E10E948C078F7180937C029E
:1017D00080E060E070E00E94170880E160E071E066
:1017E0000E94170884E162E774E00E94170880E015
:1017F0000E94EA078FE164E00E94A9071F91089503
:10180000CF93DF93EC0181E00E94EA0789E10E9417
:101810008C07882321F40E94EA0780E044C080E01E
:101820000E94EA0760917A0270917B0280E00E9438
:10183000C40780917A0290917B0290937902809301
:10184000780282E792E066E070E00E946E08809184
:1018500073028F7180937302809175028F718093F0
:101860007502209172023091730230937B022093B3
:101870007A0280917402909175028F5E954080F497
:1018800089E1283D380760F420FD0AC08091770285
:1018900087FD06C08091760284FD02C087FD06C0E8
:1018A0000E94500B82E0DF91CF910895F8948091CF
:1018B000C2059091C305A091C405B091C505809360
:1018C000730490937404A0937504B093760480918C
:1018D000C0059091C10590937C0480937B0478941B
:1018E000CE016EE070E00E946E0881E0DCCF98B11E
:1018F0008F70907F892B88B90895449898B18F7024
:10190000907F892B88B90000459A86E090E00E947C
:10191000700D459808951F93182F88B1912F9295B7
:101920009F70807F982B98B9459A86E090E00E943E
:10193000700D459888B11F70807F812B88B9459ABA
:1019400086E090E00E94700D45981F910895449A9A
:101950000E948B0C089544980E948B0C08950E945D
:10196000A70C81E090E00E94700D0895CF93DF9363
:10197000EC0103C021960E94AF0C88818823D1F727
:10198000DF91CF91089580E10E94AB0C81E090E05F
:101990000E94700D0895882311F48CE001C08EE040
:1019A0000E94AB0C81E090E00E94700D089581E0F0
:1019B0000E94AB0C86E290E00E94700D08956623B1
:1019C00049F0613011F4805C05C0623011F48C5E26
:1019D00001C08C5A80680E94AB0C81E090E00E94AC
:1019E000700D08950F931F93042F0E94DF0C10E0D9
:1019F00004C080E20E94AF0C1F5F1017D4F31F9148
:101A00000F910895682F80E040E10E94F20C089544
:101A1000CF93DF93EA010E94DF0C03C00E94AF0C5A
:101A20002196FE0184918823C9F7DF91CF91089513
:101A30000F931F938A010E94DF0CC8010E94B60C0D
:101A40001F910F9108951F93142F0E94DF0C812F77
:101A50000E94A70C81E090E00E94700D1F910895F4
:101A60008CE090E00E947F0D83E00E947D0C85E673
:101A700090E00E94700D83E00E947D0C81E090E078
:101A80000E94700D83E00E947D0C81E090E00E9436
:101A9000700D82E00E947D0C81E090E00E94700D4C
:101AA00088E20E94AB0C81E090E00E94700D88E01B
:101AB0000E94AB0C81E090E00E94700D81E00E94DA
:101AC000AB0C86E290E00E94700D86E00E94AB0CA9
:101AD00081E090E00E94700D8CE00E94AB0C0895B4
:101AE00028EC00002A95E9F70197D1F70895F894BA
:101AF00020916A0230916B027894C9010895AC017B
:101B0000F89420916A0230916B02789401C0A895F4
:101B1000F89480916A0290916B027894821B930BE7
:101B200084179507A0F308959091700289B1ECE6AF
:101B3000F2E0E90FF11D8095877080839F5F9370BD
:101B400090937002089590916D0280916C02982399
:101B500080916E02982380916F02982331F1913029
:101B600011F441E115C0923011F442E111C09430FA
:101B700011F443E10DC0953011F444E109C09330F4
:101B800011F445E105C0963011F040E001C046E196
:101B9000242F30E08091C805992787FD909528175C
:101BA000390729F04093C80503C01092C80540E0EA
:101BB000842F0895EF92FF920F931F93CF93DF939B
:101BC000F894E0906A02F0906B0278948701A895EF
:101BD000F894C0916A02D0916B027894CE01801B78
:101BE000910B059718F00E94940D8E010E94A30D91
:101BF000882331F4CE19DF09C95BDB4040F387E16C
:101C0000CDB7DEB7E6E00C94173D0F931F93CF934B
:101C1000DF939C01EB018A0101C0A895F999FDCFE2
:101C2000CE01B9014FE150E00E94C23D1F8E888174
:101C3000992787FD90950E94263D892B21F4CE019E
:101C4000B8010E944B3DDF91CF911F910F910895F4
:101C50000000000000000000000008952B9A2D985D
:101C6000000000000000000000002D9A90E087FFB7
:101C700002C02B9A01C02B982D9800000000000094
:101C8000000000002D9A9F5F983011F0880FEFCF71
:101C90000895F8942D9A289A8F7380680E942E0ECA
:101CA00080E020E030E02D980000000000000000FF
:101CB00000002D9A00000000000000000000220F2C
:101CC000331F1C9921608F5F803169F7932F28980B
:101CD000789480917102813021F4822F0E94202C0F
:101CE0009C01C90108951F93CF93DF9380E00E9468
:101CF000490E8050904419F481E08093710282E093
:101D00000E94490E8F5F9F4F61F012E0C0E0D1E06A
:101D1000812F0E94490E8883998322961F5F153078
:101D2000B9F7DF91CF911F9108951F1D1F1E1F1E30
:101D30001F1F1E1F1E1FCF93DF93EC012C964AE836
:101D400034D06627772736E4AEE6B1E0532F5370E0
:101D500009F01197321729F078F56A0F7B1F339538
:101D6000F3CF4CE022D0EAE2FDE130E0C8953196B5
:101D7000313011F451110A94321720F4600D711DA5
:101D80003395F4CF402D439510D02150A8F0620F29
:101D9000711D8827992748E108D015D04CE305D05C
:101DA00012D02CE302D00FD00BC03A912A91241705
:101DB000310540F00F900F906FEF7FEF8FEF9FEFA7
:101DC000DF91CF91089551E2AA1B08F4A40FA795C3
:101DD00097958795779567955A95B9F7620F711D15
:101DE000811D911D0895CF93DF93FC0120813181E6
:101DF00042815381CC27DD2757FD3CC0C9ECD5E09B
:101E00006CE33CD00882198239D00A821B8268E1D7
:101E100035D00C821D82F9012C5F3F4F67E02ED038
:101E20000C861D869F01A6E4EEE6F1E0BA2FB370A2
:101E300009F031972E173F0720F02E1B3F0BA3957B
:101E4000F3CFAA871B862E873F87EAE2FDE1AA2708
:101E5000C8953196A13011F4B1110A9420153105BD
:101E600020F020193109A395F3CFA887198623956F
:101E70002E833F83CE01DF91CF910895002470E23D
:101E8000220F331F441F551F001C061610F0061AA0
:101E900023957A95A9F70895EFEAF2E082818130DF
:101EA00041F480819181019791838083892B09F48A
:101EB00012823D9682E0E33EF80781F70895CF92C3
:101EC000DF92EF92FF920F931F936B017C018AE2E6
:101ED00090E090937E0280937D0280E00E94EA076A
:101EE00082E06DEC7FE10E94C4078FEF66E070E056
:101EF0000E94D40800E011E0C80166E070E00E9492
:101F0000BC0886E098E00E94920881E090E00E9480
:101F1000920880E098E00E94920886E00E9485087E
:101F200084E00E94850881E090E00E949208C80148
:101F300066E070E00E94BC086091DA027091DB02FA
:101F40008091DC029091DD020E94A30880E066E0AF
:101F500070E00E94D408C701B6010E94A3088CEC6F
:101F60009FE10E948D091F910F91FF90EF90DF90EC
:101F7000CF900895EF92FF920F931F93CF93DF932B
:101F80007B018C01E901E5EAF2E020E080819181AA
:101F9000A281B3818E159F05A007B10711F4922F7E
:101FA0000DC02F5F3D96243089F7CD2BF9F090912D
:101FB000D902892F8F5F83708093D9028DE0989F1B
:101FC000F0011124EB55FD4FEF012496DA0186E074
:101FD0000D9009928150E1F7E082F1820283138330
:101FE00080EB94E09387828781E08487CDB7DEB76A
:101FF000E6E00C94173DACE1B0E0E1E0F0E10C94D8
:10200000F53CCE0101966CE170E00E946E088F8174
:1020100098850E94202C4C016F85788989899A893E
:102020000E94242C5B016C01698D7A8D8B8D9C8DB7
:102030000E94242C7B018C0189819A810E94202C92
:10204000019709F071C08B819C810E94202C8050E7
:10205000984009F069C08091DA029091DB02A0916A
:10206000DC02B091DD02E816F9060A071B0709F049
:102070005BC0CE01439660E071E046E050E00E9414
:10208000A53D009709F050C0AE14BF04C006D106AC
:1020900011F482E04AC08E01075F1F4FC601B501EF
:1020A000A80121E030E00E94BA0F81E08816910477
:1020B000D9F58CE190E090937E0280937D028EE0D2
:1020C00090E00E94570981E090E00E94920880E031
:1020D00098E00E94920886E00E94850884E00E94B1
:1020E000850882E090E00E94920880E091E066E03E
:1020F00070E00E94BC086091DA027091DB0280916E
:10210000DC029091DD020E94A308C80166E070E045
:102110000E94BC08CE010F9664E070E00E94BC08EB
:1021200086E098E00E94031180E06C96ECE00C944D
:10213000113DEF92FF920F931F93E0908502F09074
:10214000860200918702109188022091DE02309170
:10215000DF024091E0025091E102DA01C9018E29CB
:102160009F29A02BB12B8F5F9F4FAF4FBF4F49F4DB
:102170008FE792E06FEF70E046E050E00E94833D11
:1021800035C08091DA029091DB02A091DC02B0911F
:10219000DD028E259F25A027B12782239323A42328
:1021A000B5230097A105B10511F421E009C0E09025
:1021B000E202F090E3020091E4021091E50222E0D5
:1021C000E5EAF2E08485813099F480819181A281F1
:1021D000B3818E159F05A007B10751F4AFE7B2E0B8
:1021E000349686E001900D928150E1F720E005C021
:1021F0003D9682E0E93DF80729F7822F1F910F9164
:10220000FF90EF9008950F931F938C0180917D02B2
:1022100090917E020E9690937E0280937D0280E0E4
:1022200090E00E9457098FE792E066E070E00E941C
:10223000BC0880E091E066E070E00E94BC08C80144
:102240000E94920888ED99E10E948D091F910F91DB
:102250000895AEE0B0E0EFE2F1E10C94FE3CCE0177
:1022600001960E94000C8823F1F0AFE7B2E0FE0176
:10227000379686E001900D928150E1F78D859E851D
:102280000E94202C28E08030920711F411E00CC04D
:102290008650984031F40E94FB0F182F0E9471095C
:1022A00003C00E94710910E0812F2E96E3E00C9488
:1022B0001A3DA8E0B0E0EFE5F1E10C94FD3C60913F
:1022C0007D0270917E0282E290E00E94810A892B59
:1022D00011F087E065C082E290E00E943209CE01F1
:1022E000019668E070E00E946E0899819093E9027F
:1022F0008A818093EA02983031F16D817E818F81ED
:1023000098850E94242C9B01AC016093EB02709392
:10231000EC028093ED029093EE028091E90283300B
:1023200019F40E94500B3BC08530C9F58091EA0238
:102330008130A9F52093E2023093E3024093E40256
:102340005093E5022CC040917D0250917E0282E2C2
:1023500090E062E270E00E94AB0A82E290E00E94AC
:10236000570980E00E94850880E00E94850880E08F
:1023700090E00E94920860917D0270917E0282E25C
:1023800090E00E94900A8C0184E290E00E9457093C
:10239000C8010E94920881E00E942E1201C08AE0CA
:1023A0002896E4E00C94193DA0E0B0E0EAEDF1E1FC
:1023B0000C94F83CB82EEB016A01E9E9F2E0EE2456
:1023C000FF248701308121813296C901A0E0B0E06D
:1023D000E80EF91E0A1F1B1F82E0E53AF80791F785
:1023E00081E0B81651F480E00E94EA07C752D64E49
:1023F00080E0BE010E94C40703C0CE010E943209E2
:10240000C6010E942B0A9C0140E050E02E0D3F1DAA
:10241000401F511F203080E0380781E0480780E0EE
:102420005807A0F0CA0140E050E0A0E0B0E0280F5B
:10243000391F4A1F5B1F203080E0380781E04807C2
:1024400080E0580718F0C90101969C01209530954D
:10245000C901CDB7DEB7E9E00C94143DACE1B0E0C2
:10246000E4E3F2E10C94FD3C182F80917D02909101
:102470007E02449690937E0280937D028EE090E0EF
:102480000E94570980E095E40E94920880917D02A5
:1024900090917E020E9492088091E6029091E7025C
:1024A0000E94920880E090E40E94920880E40E94DA
:1024B0008508812F0E94850880E090E00E949208A4
:1024C0006091DA027091DB028091DC029091DD0272
:1024D0000E94A30860918502709186028091870214
:1024E000909188020E94A3088EE090E064E170E081
:1024F0000E94900A8C0188E190E00E945709C8016F
:102500000E9492080E949910882309F443C0DE01BA
:102510001196EDE7F2E09CE101900D929150E1F708
:10252000823049F46091E2027091E3028091E4020A
:102530009091E50208C060918502709186028091B9
:102540008702909188020E945F0F0E9471090E9489
:10255000770D8C01A8950E942911882311F00E9403
:1025600071090E949910882311F420E008C00E948C
:10257000770D801B910B8C52914060F326E0ADE704
:10258000B2E0FE0131968CE101900D928150E1F7AD
:10259000222329F480E098E00E94031120E080913A
:1025A000E6029091E70201969093E7028093E6029B
:1025B000822F6C96E4E00C94193DA4E1B0E0E3EEC8
:1025C000F2E10C94FB3C0E942911882309F4A1C07C
:1025D000823011F485E09DC08EE090E064E170E00F
:1025E0000E94810A892B09F091C08EE090E00E9440
:1025F0003209CE01019664E170E00E946E0869899B
:102600007A898B899C890E94242C7B018C012091E2
:10261000DE023091DF024091E0025091E1028981B7
:10262000682F70E0CB01807F90708034910509F0B5
:102630006DC08091DA029091DB02A091DC02B09132
:10264000DD02E816F9060A071B0799F02E293F2933
:10265000402B512B2F5F3F4F4F4F5F4F51F08FEF6C
:10266000E8168FEFF8068FEF08078FEF180709F0CD
:102670004DC06F707070660F771F660F771F609385
:10268000E8028B819C810E94202C2091E802821B11
:10269000910990937E0280937D026D857E858F8562
:1026A00098890E94242C60938502709386028093FF
:1026B000870290938802E0928902F0928A02009346
:1026C0008B0210938C028091E802853120F08451B6
:1026D00090E00E941C0B60918502709186028091AF
:1026E0008702909188024FE752E020E030E00E949C
:1026F000BA0F8A85813011F482E00BC0813111F468
:1027000083E007C0863011F484E003C00E947109A1
:1027100080E06496E6E00C94173DA0E0B0E0E3E9C9
:10272000F3E10C94FA3CD82EEB017A0184E190E0BD
:10273000E80EF91EF0927E02E0927D028CEE9FEF91
:10274000E80EF91E82E290E00E9457098D819E8179
:102750000E9492088F8198850E94920869857A85E7
:102760008B859C850E94A3086D857E858F859889C1
:102770000E94A30880E50E9485088D2D8F730E941A
:10278000850884EB95E00E94920860E070E080E0AC
:1027900090E00E94A3086091DA027091DB028091C0
:1027A000DC029091DD020E94242C609399027093C8
:1027B0009A0280939B0290939C0269817A818B811B
:1027C0009C810E94242C60939D0270939E028093B2
:1027D0009F029093A0021092A10286E08093A20231
:1027E00080917D0290917E020E94202C9093A40201
:1027F0008093A30240917D0250917E0281E062E2CB
:1028000070E00E94D4118C0182E390E00E9457098D
:10281000C8010E94920886E00E942E12682F882329
:1028200011F58D2D992787FD909583709070892BD8
:1028300041F089859A85AB85BC850196A11DB11DA6
:102840000EC0E114F10479F0970140E050E0898571
:102850009A85AB85BC85820F931FA41FB51F8987FE
:102860009A87AB87BC87862FCDB7DEB7E7E00C949D
:10287000163DA2E1B0E0EFE3F4E10C94FF3C2091BF
:102880008D0230918E02C901A0E0B0E08A839B8363
:10289000AC83BD8380918F02909190029F838E8341
:1028A000398728871A861B861C861D86809195028B
:1028B00090919602A0919702B09198020196A11D65
:1028C000B11D8E879F87A88BB98B84E0BE016F5F97
:1028D0007F4F40E050E00E948D136296E2E00C943E
:1028E0001B3DA8E0B0E0E7E7F4E10C94F53C7C0187
:1028F00080919102909192020E94320900E010E0D2
:102900006E010894C11CD11C2BE1A22E24E0B22E32
:10291000AE0CBF1C92E0892E9924939453C0C6013B
:1029200065E070E04AE00E94010B080F191FC60124
:1029300065E770E00E94423D892B91F4E114F104B7
:1029400019F087E993E002C087E193E06BE770E05C
:102950004AE00E94010B080F191FF501908232C056
:10296000C60160E770E044E050E00E945B3D892BC7
:1029700019F4F501808226C089818D30E1F48A81C5
:102980008A30C9F480919302909194020817190734
:10299000C8F0EE0CFF1C87E194E0E80EF91E81E020
:1029A00090E0F7019183808315C00F5F1F4F0E9455
:1029B00033088A3039F0809193029091940208177D
:1029C000190798F3809193029091940208171907C0
:1029D00008F4A5CF2896ECE00C94113DCF93DF933B
:1029E000EC01009719F027E933E002C027E133E05A
:1029F000FE01EE0FFF1FDF0143E0AA0FBB1F4A9548
:102A0000E1F7AE0FBF1FA151BD4F1C9211961D9251
:102A10001D921D921C92149716961C921E92159749
:102A200018961C921E9217971D961D921D921D922C
:102A30001C92509780E8D9011D928A95E9F7E95ECA
:102A4000FB4F11821082C55EDB4F1882DF91CF9160
:102A50000895A6E2B0E0EFE2F5E10C94F13C0091BC
:102A6000E80210E0025F1F4FCE01439664E170E080
:102A70000E946E088B899C890E94202C90938E0264
:102A800080938D028D899E890E94202C90939002C4
:102A900080938F026F89788D898D9A8D0E94242C66
:102AA0006093950270939602809397029093980298
:102AB0002F8D2695269530E0C801820F931F9093A5
:102AC00092028093910280917D0290917E02821BFE
:102AD000930B90939402809393026091850270917E
:102AE000860280918702909188020E94242C609334
:102AF000990270939A0280939B0290939C0260913A
:102B0000890270918A0280918B0290918C020E94BE
:102B1000242C60939D0270939E0280939F02909359
:102B2000A0021092A10286E08093A20280917D0211
:102B300090917E020E94202C9093A4028093A30285
:102B400040917D0250917E0280E0B8010E94D41134
:102B5000892B09F099C198A1992309F495C1609036
:102B60008502709086028090870290908802E090A3
:102B70008D02F0908E02A0908F02B09090020FEE26
:102B800012E0CC24DD246FEF7FEF2E010894411C6E
:102B9000511CD201F80182E101900D928150E1F7C0
:102BA000AE81BF81E885F9852A813B814C815D81B9
:102BB0008981882331F48FEF6F3F780711F4B601D4
:102BC0000BC0261537054805590531F4EE15FF05EC
:102BD00019F4AA15BB05C1F00894C11CD11C0E5EE6
:102BE0001F4FE2E0CE16D104A1F6FFEF6F3F7F0743
:102BF00041F06B01C094D0948CE9C8168FEFD806D1
:102C000019F40E943914FFC0D7FE47C091FF3FC19D
:102C10008091130390911403A816B90609F037C1E7
:102C2000C094D094C601880F991F8C0143E0000F17
:102C3000111F4A95E1F7080F191F01511D4FF801A7
:102C40006182728283829482B682A582F086E78254
:102C500081E080830E94AF2BF801618772878387B0
:102C600094878091950290919602A0919702B091DD
:102C700098020196A11DB11D85879687A787B08B05
:102C80008CE3818B82E1B80140E050E00E948D131B
:102C9000F82E882309F4FCC053C091FF03C00E94A2
:102CA00039144DC092FF0FC0B601660F771FCB01DC
:102CB00023E0880F991F2A95E1F7680F791F61516A
:102CC0007D4F84E038C090FF3FC0C601880F991F38
:102CD0008C01B3E0000F111FBA95E1F7080F191F1F
:102CE00001511D4FF801208180919502909196022B
:102CF000A0919702B09198020196A11DB11D858700
:102D00009687A787B08B223079F480E1B80140E044
:102D100050E00E948D1381E1B80140E050E00E9434
:102D20008D13F82E85E0A1C0233019F0263009F06C
:102D3000AEC080E1B80140E050E00E948D13F82E53
:102D4000C6010E94EE14A4C093FF5FC0809193025D
:102D500090919402009711F480E055C05601AA0C9E
:102D6000BB1C8501F3E0000F111FFA95E1F70A0D76
:102D70001B1D01511D4FF8012081213019F482E003
:102D8000808302C0223011F0FF243CC0A0E0B0E0FC
:102D900020919502309196024091970250919802AD
:102DA000820F931FA41FB51FF80185879687A787F9
:102DB000B08B2581368180911303909114032817DD
:102DC0003907B1F480E1B80140E050E00E948D1372
:102DD000F82EC6010E947114F501E95EFB4F808157
:102DE0009181019779F4C6010E94422EF82E0AC003
:102DF00081E1B80140E050E00E948D13F82E83E09D
:102E0000F80180838F2DF82E43C094FF40C0C60187
:102E1000880F991F8C0173E0000F111F7A95E1F75D
:102E2000080F191F01511D4FF8018081813011F4E5
:102E300082E022C08230E1F480919302909194026A
:102E4000892B59F080E1B80140E050E00E948D13D9
:102E5000F82EC6010E9471141BC081E1B80140E048
:102E600050E00E948D13F82E83E0F801808310C09B
:102E7000833021F486E0F801808309C0853039F47D
:102E8000C6010E94EE1403C068E0F62E01C0FF24C4
:102E90008F2DA696E0E10C940D3DCF93DF9308961D
:102EA00090937E0280937D0282E290E00E94570917
:102EB00080918F02909190020E94920880918D02E1
:102EC00090918E020E94920880917D0290917E02E4
:102ED0000E94920880E090E00E9492086091DA02DD
:102EE0007091DB028091DC029091DD020E94242C23
:102EF0006093990270939A0280939B0290939C0234
:102F0000609185027091860280918702909188027B
:102F10000E94242C60939D0270939E0280939F02D6
:102F20009093A0021092A10281E18093A20280916D
:102F30007D0290917E020E94202C9093A4028093A7
:102F4000A30240917D0250917E0281E062E270E036
:102F50000E94D411EC01009711F4CFEFDFEF88E26B
:102F600090E00E945709CE010E94920881E10E94E0
:102F70002E12DF91CF910895A8E0B0E0E2ECF7E1E6
:102F80000C94FB3CCE01019668E070E00E946E0854
:102F900089819A810E94202C90938E0280938D02C9
:102FA0008B819C810E94202C9093900280938F02B1
:102FB0008D819E810E94202C7C0188EF9FEFE80E7E
:102FC000F91EF0929402E092930288E090E0E80EFD
:102FD000F91E8091E802082F10E0025F1F4F8F81D9
:102FE0009885892BC1F1609185027091860280914C
:102FF0008702909188020E94242C6093990270931A
:103000009A0280939B0290939C0260918902709136
:103010008A0280918B0290918C020E94242C6093F2
:103020009D0270939E0280939F029093A002109243
:10303000A10281E18093A2028D819E819093A402DE
:103040008093A30280E0B801A7010E94D411892BCC
:1030500011F089E024C0085F1F4F10939202009383
:10306000910280918F02909190028B37910519F413
:103070000E94972314C024E08030920719F40E9424
:10308000EF1D0DC08434910519F40E94B51B07C0D3
:103090008938910511F080E002C00E94371F289600
:1030A000E6E00C94173D8091930490919404A091D4
:1030B0009504B09196048093850290938602A09324
:1030C0008702B093880283E490E090938E0280930D
:1030D0008D0284E490E09093900280938F028AE2C4
:1030E00090E00E94570960E076E081E091E00E9464
:1030F000A3080E94AF2B6093A7047093A804809349
:10310000A9049093AA040E94A30880E090E00E9482
:10311000920880E090E00E94920860E070E080E019
:1031200090E00E94A30880E06CE070E00E94D40868
:1031300080E091E066E070E00E94BC0880E06AEC0C
:1031400070E00E94D40863E673E582E893E60E948B
:10315000A30881E095E30E94920884E00E9485081C
:1031600082E30E94850884E00E9485086091DA026B
:103170007091DB028091DC029091DD020E94A30835
:1031800086E30E94850884E00E948508609193048C
:103190007091940480919504909196040E94A308E4
:1031A0008FEF0E94850880E06CE270E00E94D408F6
:1031B0008CE291E00E944D1708950F931F9381E0D8
:1031C0008093BE048FEF9FEFAFEFBFEF8093850238
:1031D00090938602A0938702B093880283E490E0E4
:1031E00090938E0280938D0284E490E090939002FD
:1031F00080938F021092DE021092DF021092E002A2
:103200001092E1021092DA021092DB021092DC02BC
:103210001092DD021092A3051092A4051092A5054C
:103220001092A6051092E2021092E3021092E402BC
:103230001092E50210928F04109290041092910463
:103240001092920410928B0410928C0410928D04B0
:1032500010928E0410929704109298041092990480
:1032600010929A0410929304109294041092950470
:10327000109296041092A3041092A4041092A50434
:103280001092A60410929B0410929C0410929D042C
:1032900010929E0410929F041092A0041092A10418
:1032A0001092A2041092B3041092B4041092B504C8
:1032B0001092B6041092C1040E94AF2B6093A70431
:1032C0007093A8048093A9049093AA048AE290E0E2
:1032D0000E94570960E076E081E091E00E94A30837
:1032E0006091A7047091A8048091A9049091AA0408
:1032F0000E94A30860E070E880E090E00E94A308CC
:1033000080E060E170E00E94D40800E011E0C801B4
:1033100066E070E00E94BC0880E06AEC70E00E9409
:10332000D40863E673E582E893E60E94A30881E08F
:1033300095E30E94920881E00E9485088DE30E9437
:10334000850887E00E94850881E00E948508C80101
:1033500066E070E00E94BC088FEF0E94850880E064
:103360006FE270E00E94D4088CE291E00E944D1759
:103370001F910F9108950F931F93182F8093BE04F0
:10338000883129F08FEF9FEFAFEFBFEF08C080913A
:10339000930490919404A0919504B0919604809325
:1033A000850290938602A0938702B093880213301F
:1033B00051F00E94AF2B6093A7047093A8048093F0
:1033C000A9049093AA04E3E9F5E001900020E9F74D
:1033D0003197E359F5400E2F0F5F83E490E090930F
:1033E0008E0280938D0284E490E09093900280930B
:1033F0008F028AE290E00E94570960E076E081E067
:1034000091E00E94A3086091A7047091A8048091A4
:10341000A9049091AA040E94A30880E090E00E9471
:103420009208183119F080E090E802C080E090E046
:103430000E9492086091DA027091DB028091DC02B6
:103440009091DD020E94A30880E06CE070E00E9491
:10345000D40880E091E066E070E00E94BC0880E063
:103460006AEC70E00E94D40863E673E582E893E6B4
:103470000E94A30881E095E30E94920883E00E94E5
:1034800085088CE00E948508802F0E94850883E9CA
:1034900095E0602F70E00E94BC08133019F582E3BC
:1034A0000E94850884E00E94850880919102909195
:1034B000920240960E9432090E9452080E94A3087C
:1034C00086E30E94850884E00E9485086091930449
:1034D0007091940480919504909196040E94A308A1
:1034E00019E115C0163111F015E211C082E30E94F6
:1034F000850884E00E9485086091870470918804A3
:103500008091890490918A040E94A3081FE187E3B7
:103510000E94850886E00E94850881E00E94850857
:1035200083E00E94850886E00E94850883E30E946C
:1035300085088AE30E9485088BE30E9485088DE355
:103540000E94850887E00E94850881E00E94850826
:1035500080E091E066E070E00E94BC088FEF0E947E
:103560008508101B80E0612F70E00E94D4088CE277
:1035700091E00E944D171F910F910895EF92FF92D5
:103580000F931F938091BF049091C004892B59F42D
:10359000ABE0B1E0EFE1F1E082E101900D9281500A
:1035A000E1F760E0DCC08091BE04813031F086310B
:1035B00021F0883111F08931D9F5E090BB04F09009
:1035C000BC0400E010E08BE091E06FE171E00E944C
:1035D000BD2CE61AF70A080B190BE092B704F0921B
:1035E000B8040093B9041093BA041E141F04100603
:1035F0001106F4F08091BE04813049F0863159F40F
:103600008091C1048F5F8093C104833018F00E94C1
:10361000DD1803C086E10E94BB19682FABE0B1E062
:10362000EFE1F1E082E101900D928150E1F701C0FC
:1036300060E0E090B304F090B4040091B504109100
:10364000B604D801C7010196A11DB11D0297A105BD
:10365000B10508F484C08091AB049091AC04A091B2
:10366000AD04B091AE042091AF043091B00440910C
:10367000B1045091B2040097A105B10591F10197F1
:10368000A109B1098093AB049093AC04A093AD045D
:10369000B093AE0421503040404050402093AF04DE
:1036A0003093B0044093B1045093B2040894E108FD
:1036B000F10801091109E092B304F092B4040093F7
:1036C000B5041093B6040097A105B10509F047C0F1
:1036D00088E10E94BB19682F882309F040C06CE084
:1036E0003EC00894E108F1080109110921153105CE
:1036F0004105510509F1DA01C9010197A109B10993
:103700008093AF049093B004A093B104B093B2043B
:10371000E092B304F092B4040093B5041093B6049D
:103720000097A105B105D9F489E10E94BB19682F62
:103730008823A9F46DE013C0E092B304F092B404BE
:103740000093B5041093B604E114F10401051105CA
:1037500031F40E94DD18682F882309F46EE0862F6B
:103760001F910F91FF90EF900895ACE1B0E0EBEB6B
:10377000FBE10C94FB3C8091BE04882309F4E2C178
:10378000873109F4DFC180919102909192028051BA
:103790009F4F0E9432090E943308182F8F3F09F46F
:1037A000C5C00E943308082F153341F4813009F059
:1037B000D0C10E9433088093BD04EDCF113071F465
:1037C000843009F0C6C10E94520860938B04709344
:1037D0008C0480938D0490938E04DDCF133071F4AC
:1037E000843008F4B6C10E94520860938F0470932D
:1037F000900480939104909392041FC0163371F447
:10380000843008F4A6C10E94520860939304709318
:10381000940480939504909396040FC01630A1F4FD
:10382000843008F496C10E94520860939704709304
:1038300098048093990490939A04043009F4ABCFD0
:10384000802F90E004976FC0133309F04BC0843091
:1038500009F0A1CF0E9452087B018C016093A30460
:103860007093A4048093A5049093A60480919F0470
:103870009091A004A091A104B091A2040097A10589
:10388000B105B1F4C801B7012BE633E040E050E0E8
:103890000E94733C28EE33E040E050E00E94B23CCE
:1038A00020939F043093A0044093A1045093A2045A
:1038B00080919B0490919C04A0919D04B0919E04E2
:1038C0000097A105B10509F066CF16950795F79405
:1038D000E794E0929B04F0929C0400939D04109363
:1038E0009E0459CF1A3371F4843009F054CF0E94EA
:1038F000520860939B0470939C0480939D04909362
:103900009E0449CF1B3371F4843009F044CF0E94E8
:10391000520860939F047093A0048093A104909335
:10392000A20439CF90E00E941C0B35CF8091910208
:103930009091920204960E9432098091BE04909167
:10394000BD048130B9F4923009F0FEC00E945208E3
:103950002091A7043091A8044091A9045091AA0491
:10396000621773078407950709F0EEC083E00E9491
:10397000BB19EBC0953009F0D3C00E9452082091CA
:10398000A7043091A8044091A9045091AA04621799
:1039900073078407950709F0D7C087E18093BE04B9
:1039A000809191029091920240960E9432090E9469
:1039B0005208AB01BC014093DA025093DB026093E2
:1039C000DC027093DD0288E090E00E94083E809166
:1039D0008B0490918C04A0918D04B0918E048093FF
:1039E000DE029093DF02A093E002B093E1028091A7
:1039F0008F0490919004A0919104B09192048093CF
:103A0000E2029093E302A093E402B093E502809176
:103A1000970490919804A0919904B0919A0480938E
:103A2000A3059093A405A093A505B093A605809146
:103A30009B0490919C04A0919D04B0919E0480935E
:103A4000AB049093AC04A093AD04B093AE0480910A
:103A50009F049091A004A091A104B091A20480932E
:103A6000AF049093B004A093B104B093B2048091DA
:103A7000A3049091A404A091A504B091A6048093FE
:103A8000B3049093B404A093B504B093B6048F5FCD
:103A90009F4FAF4FBF4F21F41092C0041092BF044C
:103AA000DE011196EDE7F2E08CE101900D9281507C
:103AB000E1F76091DA027091DB028091DC02909173
:103AC000DD020E945F0F0E9471090E94770D8C0138
:103AD000A8950E942911813019F40E94710909C02A
:103AE000823039F40E945318882381F40E94DD1833
:103AF0000DC00E94770D801B910B4E9748F381E01B
:103B000090E09093AA058093A90580E0ADE7B2E02C
:103B1000FE0131969CE101900D929150E1F715C0A4
:103B2000963091F40E9452082091A7043091A80485
:103B30004091A9045091AA0462177307840795075E
:103B400019F407C080E001C08FE06C96E6E00C94A9
:103B5000173D0E94DD18F9CFAF92BF92DF92EF922E
:103B6000FF920F931F93DF93CF930F92CDB7DEB7E2
:103B7000F82EE92E9C0159018EE2D82E0E943308BE
:103B8000982F882331F40894A108B108F501108218
:103B900019C0807C803C11F085010AC00E94330866
:103BA00011C099830E943308F80181938F01998194
:103BB000802F8A198917A8F3A90EB11CF501D1929B
:103BC0005F01DCCF8F2D9E2D0F90CF91DF911F9144
:103BD0000F91FF90EF90DF90BF90AF900895ACE40D
:103BE000B0E0E5EFFDE10C94F13C80919102909101
:103BF00092020E943209CE0101966CE070E00E94B0
:103C00006E0889819A810E94202C2091880530912C
:103C100089058217930709F06AC08D819E810E94F1
:103C2000202C6C01EE24FF243DE2A32EB12CAC0E1F
:103C3000BD1E2DE0822E912C8C0E9D1E14C0C50140
:103C40000E94AC1D0E9440088C010E944008013077
:103C5000110531F4019721F4C401B5010E949E3D84
:103C60000894E11CF11CEC14FD0448F38F81988545
:103C70000E94202C3C01EE24FF249DE2492E512C71
:103C80004C0E5D1E31C0C2010E94AC1D0E94400856
:103C90008C010E9440084C010E9452085B016C019B
:103CA0000E94400801301105D1F421E082169104F0
:103CB000B1F48430910599F40E945208AB01BC0123
:103CC00040938A0550938B0560938C0570938D0506
:103CD000CE010D96960185010E94152208C00E9412
:103CE0001C0B0894E11CF11CE614F70460F280E060
:103CF000C45BDF4FE0E10C940D3DAF92BF92DF92C9
:103D0000EF92FF920F931F93CF93DF93182F092FFA
:103D10008091A3059091A405A091A505B091A60559
:103D20008093850290938602A0938702B0938802C5
:103D300085E390E090938E0280938D0280E094E082
:103D40009093900280938F020E94AF2B709389050D
:103D5000609388058AE290E00E9457098091880567
:103D6000909189050E94920880E091E00E9492085B
:103D700081E090E00E94920880E090E00E9492082A
:103D800080E090E00E94920880E090E00E9492081B
:103D9000212F302FC901EC0140E1A42EB12C7E016E
:103DA0000E2D0C1BF701D080FEE2DF1631F0DD2076
:103DB00021F00894E11CF11CF3CF802F0E948508AC
:103DC00010E0CE01B8010E94BC080F5F1F4FA00E8B
:103DD000B11EDD2019F0E7012196E1CF80E00E94BD
:103DE000850881E090E00E94920881E090E00E94C6
:103DF0009208C50101960E944D17DF91CF911F9146
:103E00000F91FF90EF90DF90BF90AF9008951F93B8
:103E10000E943308182F11541295107F0E94330806
:103E200081548F70812B1F9108950F931F93CF930F
:103E3000DF93EC0100E0899190E00E943A3D182F59
:103E400085958595859585958F5B0E9485081F7062
:103E5000812F8F5B0E9485080F5F003161F780E042
:103E60000E948508DF91CF911F910F910895ACE1D9
:103E7000B0E0EDE3FFE10C94F13C80919102909170
:103E800092020E943209CE0101966CE070E00E941D
:103E90006E088B819C810E94202C9C018F709070F9
:103EA000892B11F082E1EEC037FF5AC089819A81D7
:103EB0000E94202C20918805309189058217930754
:103EC00009F0DFC08F8198850E94202C019711F0A6
:103ED00080E1D8C00E943308803211F081E1D2C065
:103EE0008E01035F1F4FC801902E892E2DE1E22E17
:103EF000F12CEC0EFD1E0E94071FF80181938F012B
:103F0000EE15FF05C1F71C8E0E9433080E94400881
:103F10008C010E9440087C010E9452085B016C01E8
:103F20000032110509F0ADC0F1E0EF16F10409F01F
:103F3000A8C00E9440080E9440080E945208AB019D
:103F4000BC0140938A0550938B0560938C05709358
:103F50008D05892D982D960185010E94152291C00D
:103F600020703877232B09F08CC0809193029091B8
:103F70009402C29709F085C089819A810E94202C01
:103F80004C018D819E810E94202C5C01CC24DD247B
:103F90009DE0692E712C6C0E7D1E8DE1482E512CFA
:103FA0004C0E5D1E31C00E943308803209F069C09A
:103FB00083010E94071FF80181938F01E415F50525
:103FC000C1F71C8E0E9433080E9440087C010E94A9
:103FD00040080197B1F4F0E2EF16F10451F4C30187
:103FE00063E975E00E94953D009759F400E015E8FB
:103FF0004FC081E2E816F10421F48D858A3209F47C
:1040000045C00894C11CD11CCA14DB0460F239C03D
:1040100086E090E00E94920880E090E00E94920882
:104020006091DA027091DB028091DC029091DD02F6
:104030000E94A3088EE390E021C08DE390E00E94EF
:10404000920881E00E94850883E995E06FE070E0C6
:104050000E94BC0880E00E94850880E094E00E94F5
:10406000920880E091E066E070E00E94BC0880E089
:1040700064E270E00E94D40885E790E00E944D174A
:1040800001C080E06C96E0E10C940D3D00E014E886
:104090008AE290E00E945709C4010E949208C80178
:1040A0000E94920880E090E00E94920881E090E0F7
:1040B0000E94920880E090E00E94920880E090E0E8
:1040C0000E94920880E20E948508CE010D960E940F
:1040D000151FC7010E94920881E090E00E9492089B
:1040E00068E572E080E090E00E94A308E0E2EE164E
:1040F000F10409F0A2CF8CCF0F931F938C01809114
:10410000DE029091DF02A091E002B091E102809581
:104110009095A095B0952091DA023091DB02409104
:10412000DC025091DD02822B932BA42BB52B8093C4
:10413000850290938602A0938702B093880289E853
:1041400090E090938E0280938D02909390028093E2
:104150008F020E94AF2B70938905609388058AE2D5
:1041600090E00E94570980918805909189050E94EE
:10417000920880E191E00E94920881E090E00E9424
:10418000920880E090E00E94920880E090E00E9417
:10419000920880E090E00E94920880E20E948508E8
:1041A000C8010E94151F80E290E00E94920881E001
:1041B00090E00E94920882E390E00E944D171F91C8
:1041C0000F910895E6E0F5E084818130A1F48081CB
:1041D0009181A281B3810097A105B10561F001979A
:1041E000A109B10980839183A283B3830097A105BC
:1041F000B10509F41482B99685E0EA3AF80721F787
:104200000895A9E2B0E0E7E0F1E20C94F93C7C010A
:1042100002EE14E06E010894C11CD11CD601F80115
:1042200089E201900D928150E1F789A5813059F41E
:10423000C601B7010E94953D009729F429A13AA132
:104240004BA15CA10AC0075D1F4F85E00638180727
:1042500029F720E030E040E050E0B901CA01A9961A
:10426000E8E00C94153DCF93DF9380919005813069
:1042700001F5C2ECD4E0CE016AE875E00E942A2C78
:10428000813009F4C3C0FE0101900020E9F73197A5
:10429000EC1BFD0B709738F4CE016EE270E00E94CB
:1042A0008A3D009711F084E001C082E08093900580
:1042B000A9C0823009F582EC94E00E94012160934C
:1042C0008A0570938B0580938C0590938D056115FD
:1042D00071058105910509F099C00E94770D9093B1
:1042E00087058093860582EC94E00E947C20282F2D
:1042F00010928F0583E053C0833079F580918A0551
:1043000090918B05A0918C05B0918D050097A1052A
:10431000B10509F07BC00E94770D20918605309190
:104320008705821B930B8C52914008F46BC08091DF
:104330008F058F5F80938F05833020F0209161047B
:104340002D5E61C00E94770D90938705809386054E
:1043500082EC94E00E947C2053C0843019F582ECFA
:1043600094E00E94012160938A0570938B058093ED
:104370008C0590938D05611571058105910509F0F6
:1043800045C00E94770D909387058093860582EC47
:1043900094E00E947D1E282F10928F0585E0809367
:1043A000900531C0853071F580918A0590918B051B
:1043B000A0918C05B0918D050097A105B10531F54F
:1043C0000E94770D2091860530918705821B930B03
:1043D0008C529140B8F080918F058F5F80938F054C
:1043E000833020F020916104295E0DC00E94770D7A
:1043F000909387058093860582EC94E00E947D1E51
:10440000282F01C020E080E090E003C020E081E0A0
:1044100090E09093920580939105019711F410928A
:104420009005822FDF91CF910895A0E0B0E0EBE1FD
:10443000F2E20C94F53CEC016A017B014801590160
:1044400082EE94E0BE010E94953D0097B9F18BE0A9
:1044500095E0BE010E94953D009781F184E395E0CF
:10446000BE010E94953D009749F18DE595E0BE01A2
:104470000E94953D009711F120918E05822F8F5F4C
:10448000837080938E0530E089E290E0289F800160
:10449000299F100D389F100D11240E511B4FC8017C
:1044A000BE010E949E3DF801C0A2D1A2E2A2F3A2E9
:1044B00084A295A2A6A2B7A281E080A7CDB7DEB75D
:1044C000ECE00C94113DA8E0B0E0E9E6F2E20C94D7
:1044D000F73C6D837E838F83988719821A821B82B3
:1044E0001C8229813A814B815C81ECE2AE2EBB2497
:1044F000B394CC24DD24EE24FF2400E010E00E94DD
:10450000FE35952FB901842F2896EAE00C94133DCF
:10451000A0E2B0E0EEE8F2E20C94FB3C7C01E62F76
:10452000F0E0EE0FFF1FE155FF4F659174918E0192
:104530000F5F1F4FC8010E949E3DC801B7010E9436
:104540002A2CA096E6E00C94173DA4E0B0E0EBEA3C
:10455000F2E20C94FB3C109161041093620400E0C1
:104560007E010894E11CF11C1F5F1370C701612FCD
:104570000E948822813041F489819A81AB81BC817B
:104580000097A105B10519F01093610403C00F5FF6
:10459000043051F72496E6E00C94173DAF92BF9299
:1045A000CF92DF92EF92FF920F931F936093850259
:1045B0007093860280938702909388028BE790E045
:1045C00090938E0280938D029093900280938F023D
:1045D0008AE290E00E94570983E20E94850880E009
:1045E00067E270E00E94D408F894E090C205F09071
:1045F000C3050091C4051091C5056091C005709177
:10460000C105882777FD8095982F0E9463225B0162
:104610006C01789460936F047093700480937104BC
:104620009093720480E89EE7AAEAB3E8E80EF91EC8
:104630000A1F1B1FC801B7010E94A308C601B501CC
:104640000E94A30880E390E00E944D171F910F91F4
:10465000FF90EF90DF90CF90BF90AF9008951F93A1
:104660001091B005112309F45EC01130A1F48091BE
:104670006104E82FF0E0EE0FFF1FE155FF4F659159
:10468000749182EC94E00E949E3D1093900582E02C
:104690008093B00548C0123079F5809191059091D2
:1046A0009205019709F03FC0109292051092910572
:1046B00060918A0570918B0580918C0590918D0594
:1046C00060931D0470931E0480931F049093200434
:1046D0000E94CE22182F882351F483E08093B005E6
:1046E0000E94770D9093800480937F0402C0109203
:1046F000B0050E94A52218C01330A9F40E94770DBE
:1047000020917F0430918004821B930B20918104BF
:10471000309182048217930730F0109306011091B4
:104720006204145E01C010E0812F1F910895A9E575
:10473000B0E0EDE9F3E20C94EF3C809191029091AE
:1047400092020E943209CE01819660E370E00E94DD
:104750006E0899A1892F8770843009F0D7C38091A2
:10476000B005882309F454C7907C909307019AA15F
:10477000892F81508F3048F082E08093060110929B
:1047800090051092B0058BE144C79F5F909308019C
:104790006DA17EA18FA198A50E94242C609367042F
:1047A000709368048093690490936A0469A57AA55C
:1047B0008BA59CA50E94242C60936B0470936C04C1
:1047C00080936D0490936E04FE01E05CFF4F908136
:1047D0002FAD5EAD6DAD7CADABADDAAC99ACFE018D
:1047E000EC5BFF4FC080FE01ED5BFF4FB080FE0130
:1047F000EE5BFF4FA080FE01EF5BFF4F7080FE017C
:10480000E85BFF4F8081FE01E95BFF4F3081FE01D5
:10481000EA5BFF4F4081FE01EB5BFF4FE081E82E3A
:10482000E91A91E08E1508F090E0832F821B21E0B9
:10483000381708F020E0F82EF91A91E08F1508F0EB
:1048400090E0292B842F851B31E0481708F030E0D9
:10485000082F021B91E0801708F090E0392B8E2F73
:10486000861B21E0E81708F020E0182F131B91E0C9
:10487000811708F090E0292B8C2D871B31E0C8169A
:1048800008F030E0B82FB21B91E08B1708F090E0F1
:10489000392B8B2D8A1B21E0B81608F020E0A82FB9
:1048A000A31B91E08A1708F090E0292B8A2D8D191F
:1048B00091E0A81608F090E0F82FF21B21E08F1786
:1048C00008F020E0922BE72DE919E91B9701A801D8
:1048D0006B2F7A2F8F2F9E2F52F52E2D2F5F81E079
:1048E0002E1508F080E0382F3F0D81E03F1508F0CD
:1048F00080E0482F400F81E0401708F080E0582FFB
:10490000510F81E0511708F080E0682F6B0F81E0B4
:104910006B1708F080E0782F7A0F81E07A1708F0A3
:1049200080E08F0F91E08F1708F090E09E0F01E07C
:104930000E947935622E532E442E352E262E6696F1
:104940007FAF669767968FAF679768969FAF6897B8
:10495000FE01E45BFF4FC080FE01E55BFF4FB080CE
:10496000FE01E65BFF4FA080FE01E75BFF4F70801A
:10497000FE01E05BFF4F0081FE01E15BFF4FF08035
:10498000FE01E25BFF4F9080FE01E35BFF4F808002
:104990008091730490917404A0917504B091760491
:1049A00080589148A545BC47182F8D8B9E8BAF8BA7
:1049B000B88F60917B0470917C0480E090E00E944D
:1049C0006322698B7A8B8B8B9C8B872F3B89492F3A
:1049D0005E897F89E88DD02ED61A91E00D1508F0FA
:1049E00090E02F2D281B822F21E0F81608F020E000
:1049F000E82EE91A91E08E1508F090E0292B892D18
:104A0000831B31E0981608F030E0F82EF21A91E09E
:104A10008F1508F090E0392B882D841B21E0881633
:104A200008F020E0082F031B91E0801708F090E0C9
:104A3000292B3C2D311B132F91E0C31608F090E079
:104A4000B12FB21B81E01B1708F080E0982B8B2D53
:104A5000851B21E0B81608F020E0A82FA91B91E0E3
:104A60008A1708F090E0292B8A2D871B91E0A81661
:104A700008F090E0F82FF21B21E08F1708F020E0FB
:104A8000922B7E1AE72DE91B2D2D3E2D4F2D502FF9
:104A90006B2F7A2F8F2F9E2F52F52D2D2F5F81E0B8
:104AA0002D1508F080E0382F3E0D81E03E1508F00E
:104AB00080E0482F4F0D81E04F1508F080E0582F1F
:104AC000500F81E0501708F080E0682F6B0F81E0F5
:104AD0006B1708F080E0782F7A0F81E07A1708F0E2
:104AE00080E08F0F91E08F1708F090E09E0F01E0BB
:104AF0000E947935A32FB42F152F062FF72ED82E0D
:104B0000C22EC60CF1E0C21608F0F0E03A2F350DC7
:104B1000E1E03A1708F0E0E0EF2EE30E21E0E316C3
:104B200008F020E0E22B4B2F440D31E04B1708F04A
:104B300030E0AE2FA40F21E0A41708F020E0322BC4
:104B4000512F530D41E0511708F040E0F32FF50FBE
:104B500021E0F51708F020E0422B602F620D31E0D4
:104B6000601708F030E0E42FE60F21E0E61708F0C8
:104B700020E0322B66967FAD66977F0D41E07F1572
:104B800008F040E0532F570F21E0571708F020E0BE
:104B9000422B67968FAD67978D0D21E08D1508F03C
:104BA00020E0480F31E0481708F030E0232B6896EA
:104BB0008FAD6897980F290FC98AEA8AAB8BFC8B57
:104BC000ED8B5E8B4F8B288F6D887E888F88988CBD
:104BD000A988BA88CB88DC889501A60160E070E0DE
:104BE00080E090E002E00E94FA34122FF32EE42ECF
:104BF000D52EC62EA72E582E392E0E94FA34B22E4C
:104C0000B10E21E0B11608F020E03F0DE1E03F15C4
:104C100008F0E0E0422E430E21E0431608F020E0C9
:104C2000E22B4E0D31E04E1508F030E0EE2EE40E92
:104C300021E0E41608F020E0322B5D0D41E05D1527
:104C400008F040E0D32ED50E21E0D51608F020E084
:104C5000422B6C0D31E06C1508F030E0C42EC60E0E
:104C600021E0C61608F020E0322B7A0D41E07A15DB
:104C700008F040E0A32EA70E21E0A71608F020E0E0
:104C8000422B850D21E0851508F020E0542E580EAA
:104C900031E0581608F030E0232BF32CF90EF20E19
:104CA0002B2D342D4E2D5D2D6C2D7A2D852D9F2D88
:104CB00004E00E94FA34A32FB42F052F162F372EAD
:104CC000282EE22FEB196996EFAF6997F1E02E17C6
:104CD00008F0F0E03A2F3419E1E0A31708F0E0E023
:104CE000B32EBF1A21E03B1508F020E0E22B4B2F3A
:104CF0004E1931E0B41708F030E0A42FAE1B21E0CC
:104D00004A1708F020E0322B502F5D1941E00517BB
:104D100008F040E0F52FF31B21E05F1708F020E0DA
:104D2000422B612F6C1931E0161708F030E0E62FA6
:104D3000E41B21E06E1708F020E0322B732D7A1966
:104D400041E0371608F040E0572F531B21E075175C
:104D500008F020E0422B822D851921E0281608F06A
:104D600020E0382F341B432F31E0841708F030E067
:104D7000232B9F19921B69968FAD6997898FBA8EE5
:104D8000AB8FFC8FED8F5E8F4F8F98A3ED8CFE8CD9
:104D90000F8D18A180911D0190911E01892B09F59D
:104DA000609185047091860461157105D1F0809140
:104DB000B3059091B405892BA1F4A401930197FE4A
:104DC00007C022273327A90126193709480959099D
:104DD000CB01A0E0B0E082179307A407B5070CF45D
:104DE00017C497011092B4051092B305F8948091FE
:104DF000C2059091C305A091C405B091C505860D6B
:104E0000971DA81DB91D8093C2059093C305A0935B
:104E1000C405B093C5058091C0059091C1058E0D64
:104E20009F1D9093C1058093C0058091C00590910E
:104E3000C10597FF2AC08091C2059091C305A0913A
:104E4000C405B091C505181619061A061B06ECF420
:104E50008091C2059091C305A091C405B091C5058C
:104E60000197A109B1098093C2059093C305A0934E
:104E7000C405B093C5058091C0059091C1058851C6
:104E80009C4F9093C1058093C0058091C20590917D
:104E9000C305A091C405B091C50580937704909394
:104EA0007804A0937904B0937A048091C00590911E
:104EB000C10590937E0480937D04789497FE0AC088
:104EC000121613063CF40894611C711C811C911C81
:104ED000285E3340D401C30180509048AF4FBF4F8C
:104EE00080509040A140B04038F08FEF9FE7909302
:104EF00064048093630404C0709264046092630449
:104F0000309366042093650481E080C3833009F008
:104F1000F1C0292F28738091B1059091B2050197B6
:104F2000F1F550900701522A40900801E090770473
:104F3000F09078040091790410917A0480E89EE75B
:104F4000AAEAB3E8E80EF91E0A1F1B1F60917D0450
:104F500070917E0480E090E00E9463223B014C014E
:104F6000A0907304B0907404C0907504D09076043F
:104F700080E89EE7AAEAB3E8A80EB91ECA1EDB1EA7
:104F800060917B0470917C0480E090E00E94632239
:104F900065966CAF7DAF8EAF9FAF659713C030EC59
:104FA000532E522A65961CAE1DAE1EAE1FAE6597DF
:104FB000662477244301AA24BB246501EE24FF2440
:104FC000870144248AE290E00E945709852D84607D
:104FD0000E948508842D0E9485088BA10E94850867
:104FE00086EF0E94850860E070E080E090E00E941B
:104FF000A30860E070E080E090E00E94A308609168
:10500000DA027091DB028091DC029091DD020E9455
:10501000A308C801B7010E94A308C401B3010E94FC
:10502000A3088091B1059091B205019799F4CE0142
:1050300081968C01085D1F4F20E3E22EF12CE80ED3
:10504000F91ED8018D918D010E9485080E151F054E
:10505000C1F70CC060E070E080E090E00E94A3081F
:1050600060E070E080E090E00E94A308C601B50116
:105070000E94A30865966CAD7DAD8EAD9FAD659722
:105080000E94A3088091B1059091B205019739F073
:10509000AA24BB246501EE24FF2487011EC0F894D6
:1050A000E090C205F090C3050091C4051091C505BC
:1050B00080E89EE7AAEAB3E8E80EF91E0A1F1B1F64
:1050C0006091C0057091C105882777FD8095982F64
:1050D0000E9463225B016C017894C801B7010E94B1
:1050E000A308C601B5010E94A30880E390E00E94D6
:1050F0004D178FC2853009F08BC2907C90930701C9
:105100009AA1892F81508F3008F082C29F5F9093BF
:1051100008016DA17EA18FA198A50E94242C609307
:105120006704709368048093690490936A0469A586
:105130007AA58BA59CA50E94242C60936B04709388
:105140006C0480936D0490936E04FE01E05BFF4F4E
:10515000D080FE01E15BFF4FC080FE01E25BFF4FAC
:10516000A080FE01E35BFF4F10813D2DD9822C2DE5
:10517000CA829A2DAB82812F1C83FE01E45BFF4F14
:10518000D080FE01E55BFF4FC080FE01E65BFF4F74
:10519000A080FE01E75BFF4F1081DD82CE82AF82EF
:1051A0001887032FF22EE92EB82E832F822B892BFE
:1051B0008B298D298C298A29812B09F429C2F894FD
:1051C0008091C2059091C305A091C405B091C50519
:1051D00080589148A545BC478D839E83AF83B8878F
:1051E0006091C0057091C105882777FD8095982F43
:1051F0000E94632269837A838B839C83789489815C
:105200002A813B814C815D81AE81BF819884F02FE2
:10521000F81B91E00F1708F090E08F2D821B21E022
:10522000F81608F020E0E82FE91B91E08E1708F04F
:1052300090E0292B8E2D831B31E0E81608F030E03A
:10524000782F721B91E0871708F090E0392B8B2D97
:10525000841B21E0B81608F020E0682F631B91E062
:10526000861708F090E0292B8D2D851B31E0D8168C
:1052700008F030E0582F521B91E0851708F090E0BD
:10528000392B8C2D8A1B21E0C81608F020E0482F0E
:10529000431B91E0841708F090E0292B8A2D8B1B8B
:1052A00091E0A81608F090E0382F321B21E0831718
:1052B00008F020E0922B1919191BF983EA837B83EC
:1052C0006C835D834E833F8318876D807E808F80E3
:1052D0009884A980BA80CB80DC809501A60160E02B
:1052E00070E080E090E002E00E94FA34122FF32E8A
:1052F000E42ED52EC62EA72E582E392E0E94FA3413
:10530000B22EB10E21E0B11608F020E03F0DE1E031
:105310003F1508F0E0E0422E430E21E0431608F06E
:1053200020E0E22B4E0D31E04E1508F030E0EE2E7D
:10533000E40E21E0E41608F020E0322B5D0D41E0A0
:105340005D1508F040E0D32ED50E21E0D51608F00B
:1053500020E0422B6C0D31E06C1508F030E0C42EDB
:10536000C60E21E0C61608F020E0322B7A0D41E08F
:105370007A1508F040E0A32EA70E21E0A71608F04A
:1053800020E0422B850D21E0851508F020E0542E09
:10539000580E31E0581608F030E0232BF32CF90EAC
:1053A000F20E2B2D342D4E2D5D2D6C2D7A2D852D4D
:1053B0009F2D04E00E94FA34A32FB42F052F162F3F
:1053C000372E282EE22FEB196A96EFAF6A97F1E09D
:1053D0002E1708F0F0E03A2F3419E1E0A31708F097
:1053E000E0E0B32EBF1A21E03B1508F020E0E22BED
:1053F0004B2F4E1931E0B41708F030E0A42FAE1B4C
:1054000021E04A1708F020E0322B502F5D1941E0CF
:10541000051708F040E0F52FF31B21E05F1708F0B7
:1054200020E0422B612F6C1931E0161708F030E0B4
:10543000E62FE41B21E06E1708F020E0322B732DDD
:105440007A1941E0371608F040E0572F531B21E04E
:10545000751708F020E0422B822D851921E02816CF
:1054600008F020E0382F341B432F31E0841708F078
:1054700030E0232B9F19921B6A968FAD6A9789871C
:10548000BA86AB87FC87ED875E874F87988BED8464
:10549000FE840F85188980911D0190911E01892B32
:1054A00009F5609185047091860461157105D1F04C
:1054B0008091B3059091B405892BA1F4A4019301C7
:1054C00097FE07C022273327A90126193709480963
:1054D0005909CB01A0E0B0E082179307A407B507F4
:1054E0000CF496C097011092B4051092B305F8948D
:1054F0008091C2059091C305A091C405B091C505E6
:10550000860D971DA81DB91D8093C2059093C305F4
:10551000A093C405B093C5058091C0059091C105C5
:105520008E0D9F1D9093C1058093C0058091C0058D
:105530009091C10597FF2AC08091C2059091C30543
:10554000A091C405B091C505181619061A061B06C8
:10555000ECF48091C2059091C305A091C405B0916F
:10556000C5050197A109B1098093C2059093C305B0
:10557000A093C405B093C5058091C0059091C10565
:1055800088519C4F9093C1058093C0058091C205BE
:105590009091C305A091C405B091C505809377048F
:1055A00090937804A0937904B0937A048091C00515
:1055B0009091C10590937E0480937D04789497FE2A
:1055C0000AC0121613063CF40894611C711C811C5D
:1055D000911C285E3340D401C30180509048AF4FE6
:1055E000BF4F80509040A140B04038F08FEF9FE710
:1055F000909364048093630404C070926404609286
:105600006304309366042093650482E08093A805C8
:1056100080E0C75ADF4FE2E10C940B3DDB01982F8D
:1056200092959F7023EB30E0F901E90FF11DE491B1
:10563000EC938F70280F311DF901849111968C9392
:10564000119712961C921297CB010895282FDB0117
:1056500064E60E94923C392F822F0E94923C805D2A
:10566000FD018193832F6AE00E94923C805D119638
:105670008C931197832F0E94923C905D91831282AC
:10568000CD010895A0E0B0E0E8E4FBE20C94FA3C20
:10569000482FF92EE62ED72E862F972F9C01E90151
:1056A000E0E1F7E200E010E0842F9F2DBF010E94AF
:1056B0009E3C262F842F9F2DBF010E949E3C482F89
:1056C000F92E205D2993CF016AE070E00E949E3C94
:1056D000FB010F5F1F4F0430110531F7405D488318
:1056E00019828E2D9D2DCDB7DEB7E7E00C94163DC7
:1056F0001F93CF93DF93EC0120E030E040E050E0D7
:105700001881812F80538A30C8F4CA01B9012AE078
:1057100030E040E050E00E94733C9B01AC01812FDF
:10572000992787FD9095C097AA2797FDA095BA2F36
:10573000280F391F4A1F5B1F2196E2CF203080E0DF
:10574000380781E0480780E0580720F02FEF3FEF4F
:1057500040E050E0C901DF91CF911F910895EF9291
:10576000FF920F931F938091590190915A01A0913C
:105770005B01B0915C017C018D017BE0EE0CFF1CB4
:10578000001F111F7A95D1F7E826F9260A271B2753
:1057900080915D0190915E01A0915F01B0916001E7
:1057A0008093590190935A01A0935B01B0935C01DF
:1057B0008091610190916201A0916301B0916401B7
:1057C00080935D0190935E01A0935F01B0936001AF
:1057D0008091650190916601A0916701B091680187
:1057E0008093610190936201A0936301B09364017F
:1057F0009C01AD0163E156954795379527956A95CC
:10580000D1F7282739274A275B272E253F25402710
:105810005127EF2CF02E012F11272E253F25402751
:10582000512720936501309366014093670150939F
:105830006801B901CA011F910F91FF90EF9008957F
:10584000282F892F922F0895362F272F692F782FF1
:10585000C9010895A0E2B0E0E0E3FCE20C94F53C5D
:105860009C015B018E010F5F1F4FC801B9010E94AF
:105870009E3DCC24DD247601980140E1842E912CBC
:105880008C0E9D1EF80180818E3291F41082C90128
:105890000E94782BA0E0B0E08C299D29AE29BF2979
:1058A000CC24D82EE92EFA2E98012F5F3F4F2BC023
:1058B0008823E9F4CE0101960817190731F4F501A0
:1058C000108211821282138210C0F8011082C90165
:1058D0000E94782BA0E0B0E08C299D29AE29BF2939
:1058E000F50180839183A283B38381E013C099275C
:1058F00087FD9095C0970A9730F0F50110821182CC
:105900001282138206C00815190519F00F5F1F4F88
:10591000B9CF80E0A096ECE00C94113DCF92DF92DD
:10592000EF92FF920F931F936B01E82E8A01892F4C
:10593000BA010E94262B5EE2F52EF801F382B8012F
:105940006C5F7F4F8E2D0E94262BF801F782B801E5
:10595000685F7F4F8D2D0E94262BF801F386B801DA
:10596000645F7F4F8C2D0E94262BC8011F910F91E1
:10597000FF90EF90DF90CF900895CF92DF92EF925B
:10598000FF920F931F936B010E949B0E7B018C0172
:10599000C6010E949B0E9B01AC012E193F09400BD2
:1059A000510BB901CA011F910F91FF90EF90DF9049
:1059B000CF900895A4E0B0E0E0EEFCE20C94FD3C52
:1059C000162F072F0E949B0E2091550130915601F2
:1059D0004091570150915801260F371F481F591FFA
:1059E00029833A834B835C83CE0101960E94F30E98
:1059F000AC01009711F480E00BC0812F902F9C0127
:105A0000D901FA0182E101900D928150E1F781E024
:105A10002496E4E00C94193D1F920F920FB60F925A
:105A200011242F938F939F93AF93BF9380916A021A
:105A300090916B02019690936B0280936A02809121
:105A4000C0059091C10501969093C1058093C00552
:105A50008091C0059091C1058C529140ECF010925C
:105A6000C1051092C0058091C2059091C305A09117
:105A7000C405B091C5050196A11DB11D8093C20555
:105A80009093C305A093C405B093C50581E090E051
:105A90009093C7058093C605BF91AF919F918F9159
:105AA0002F910F900FBE0F901F901895A8E2B0E0B5
:105AB000ECE5FDE20C94EF3C082F112707FD109553
:105AC000000F111FF801E251FD4F85919491F801EB
:105AD000E555FF4F4591549125E0A22EB12CAC0E17
:105AE000BD1EB5010E94050EF801E651FD4FE5907F
:105AF000F490F801EA52FD4FC590D4908FE993E0FD
:105B00000E942F0B9EA38DA3C7010E942F0B8C0117
:105B100081E893E00E942F0B98A78FA3C6010E94F3
:105B20002F0B1C0188E793E00E942F0B2C0181E2D0
:105B30007E010894E11CF11CB7010E94262BF7019D
:105B400001900020E9F73197EE19FF09BF010E948B
:105B5000BC083C018AE693E00E942F0B4C018FE1C8
:105B6000B7010E94262BF70101900020E9F7319739
:105B7000EE19FF09BF010E94BC086C0180E693E0AA
:105B80000E942F0B7C01F50101900020E9F731976D
:105B9000EA19FB09C501BF010E94BC082DA13EA165
:105BA000020F131F2FA138A5020F131F020D131D83
:105BB000040D151D060D171D080D191D0C0D1D1DBD
:105BC0000E0D1F1D080F191FC801A896E2E10C94C5
:105BD0000B3DA0E0B0E0EFEEFDE20C94F33C3C01A5
:105BE00086E390E00E94570985E391E00E942F0B25
:105BF0004C0184E093E00E942F0BEC0189E493E0D8
:105C00000E942F0B5C01E0E0F3E0859194910E94EB
:105C10002F0B6C018BE393E00E942F0B7C0180E043
:105C20000E94562D8C0181E00E94562DC80DD91D71
:105C3000CA0DDB1DCC0DDD1DCE0DDF1DC00FD11F2C
:105C4000C80FD91F81E06816710419F483E692E049
:105C500002C08BE992E00E942F0BC80FD91F8FE181
:105C600093E00E942F0B6091150370911603C80FEB
:105C7000D91F88E1AE010E948D13CDB7DEB7EEE0EB
:105C80000C940F3DA4E2B0E0E8E4FEE20C94F23C98
:105C90009C01880F991FBC01F3E0660F771FFA95EE
:105CA000E1F7680F791F61517D4F70931603609380
:105CB0001503F901E55EFB4FE081E13009F092C088
:105CC000232B19F007E913E002C007E113E0C80134
:105CD00068E173E00E94693DFC011082E0E0F3E0BE
:105CE00065917491C80146E050E00E945B3D892BAC
:105CF00061F0E2E0F3E065917491C80146E050E0A4
:105D00000E945B3D892B51F468C0E7E06E2E712C38
:105D1000600E711EF8018781882319F480E090E0FD
:105D200059C081E294E09A83898381E494E09C8362
:105D30008B8373E0C72ED12CCC0EDD1EEE24FF2406
:105D400065E0862E912C8C0E9D1E50E2552E42E071
:105D5000A42EB12CAE0CBF1CF501EA52FD4F65918B
:105D60007491C3010E94693D8C01009779F1F4019F
:105D7000852D11928A95E9F7B8016D5F7F4FC401B7
:105D80000E949E3DF60180819181B4010E949E3D5A
:105D9000F501E251FD4F6591749101C0A895F99903
:105DA000FDCFC40140E250E00E94E63D01501040AA
:105DB000F80110828EEF9FEFE80EF91EC80ED91E73
:105DC0009CEFE9169FEFF90609F0C1CF0E94C403CA
:105DD00081E090E00E94E92D1BC060911503709155
:105DE000160311C0E23079F486E390E00E9457096F
:105DF00084EC90E00E942F0BAC0160911503709130
:105E0000160388E103C081E140E050E00E948D1359
:105E1000A496EFE00C940E3DA4E0B0E0E2E1FFE2D6
:105E20000C94F73C5C016B01CB0160E074E00E94D4
:105E30004B3DF50181818E010F5F1F4FB8010E941C
:105E4000262B82E0E82EF12CEC0EFD1EC601B701D8
:105E500042E050E00E94B33DF5018281B8010E940A
:105E6000262BC6010396B70142E050E00E94B33DE5
:105E7000F5018381B8010E94262BC6010696B70161
:105E800042E050E00E94B33D2496EAE00C94133DBA
:105E9000AF92BF92DF92EF92FF920F931F93CF9337
:105EA000DF93D82E7B01FB01108189E06D2D0E94CC
:105EB000180DA8954A9BFDCF012F81E00E94CB0CC5
:105EC00019E0C0E0D0E091E0A92EB12C01C01F5F25
:105ED000812F6D2D0E94DF0C802F992787FD9095D3
:105EE0000C2E02C0959587950A94E2F780FD02C0BA
:105EF00080E204C0FE01E852FC4F84910E94AF0C86
:105F00000E94C30C0E94DA0D813149F4C5010C2EA8
:105F100002C0880F991F0A94E2F70827D9CF82316F
:105F200041F42196C730D10594F219E0C0E0D0E0E9
:105F3000CFCF833129F4F7010083C1E0D0E004C062
:105F4000873131F6C0E0D0E080E00E94CB0CCE017A
:105F5000DF91CF911F910F91FF90EF90DF90BF9055
:105F6000AF900895A0E0B0E0E8EBFFE20C94F63CBF
:105F7000982E6B0188E0692DA6010E94180DF6018C
:105F800010869081892F80538A3040F0892F815468
:105F9000863010F080E002C0892F8753A8954A9B75
:105FA000FDCFC82FDD27C7FDD09581E00E94CB0C27
:105FB00078E0B72EAA2400E010E08B2D692D0E9416
:105FC000DF0C60EDE62E63E0F62EE00EF11EF70129
:105FD000849190E08C179D071CF050E3A52EAC0E29
:105FE0008A2D0E94AF0C0E94C30C0E94DA0D8131F1
:105FF000A1F42196F701849190E08C179D072CF471
:1060000040E3A42EC0E0D0E003C030E3A32EAC0EEA
:10601000F601E00FF11FA082D0CF823169F50F5F4A
:106020001F4FB394F601E00FF11F8081992787FD80
:1060300090950E94263D892B19F40F5F1F4FB39452
:106040000830110524F028E0B22E00E010E0F6013F
:10605000E00FF11FE0818E2F80538A3040F08E2FA9
:106060008154863010F080E002C08E2F8753C82FF5
:10607000DD27C7FDD095A1CF833119F4C1E0D0E071
:1060800005C0873109F099CFC0E0D0E080E00E94E0
:10609000CB0CCE01CDB7DEB7EBE00C94123DA0E007
:1060A000B0E0E5E5F0E30C94FA3CEC018B01FB0178
:1060B000D08006960E94782BE82EFBE3F817B8F004
:1060C0001D82CE0103960E94782BF82E8BE38F154C
:1060D00070F01A82CE010E94782B883140F4F801CA
:1060E000D0828183F282E38221E030E002C020E0AE
:1060F00030E0C901CDB7DEB7E7E00C94163DA0E370
:10610000B0E0E5E8F0E30C94FB3C8091B5058093AA
:10611000DB058091B8059091B905A091BA05B091C1
:10612000BB058093DC059093DD05A093DE05B0935D
:10613000DF058091BC059091BD05A091BE05B09191
:10614000BF058093E0059093E105A093E205B0932D
:10615000E3050E94D70C80E060E040EE53E00E942F
:10616000080D8091DB05E82FF0E0EE0FFF1FE653EE
:10617000FC4F4591549181E061E00E94080D0E941E
:10618000DA0D8131B9F48091DB058F5F8093DB05F7
:10619000833010F01092DB0581E00E94020D8091A7
:1061A000DB05E82FF0E0EE0FFF1FE653FC4F4591B3
:1061B0005491E1CF833119F0873109F710C1109262
:1061C000B7051092B6058091DB05882309F4B2C0AB
:1061D0008E010F5E1F4F8CED95E0B8010E940C2FD1
:1061E000E1E2EE2EF12CEC0EFD1E80EE95E0B70103
:1061F0000E940C2F0E94D70C81E060E049EF53E031
:106200000E94080D88E060E0A8010E94180D80E05F
:1062100061E041EF53E00E94080D88E061E0A701D2
:106220000E94180D80E0B8010E94B22F892B09F45A
:10623000D6C0C8016CED75E00E944F30892B09F47F
:10624000CEC081E0B7010E94B22F892B09F4C7C0EC
:10625000C70160EE75E00E944F30892B09F4BFC082
:10626000B8C09091DC0548ED53E09A018E010F5FB4
:106270001F4FA0E2BE01695F7F4F90FF05C0F9018B
:106280008491F801808302C0F801A0832F5F3F4F03
:106290000617170721F095950F5F1F4FEECF188651
:1062A0002091E005DE01199630E2CD01FA2EE92EAB
:1062B000BE01615F7F4F20FF04C0FA0184918C937F
:1062C00001C03C934F5F5F4FA617B70719F02595A4
:1062D0001196F1CF188A0E94D70C80E060E043E16C
:1062E00054E00E94080D89E060E08E010F5F1F4FAF
:1062F000A8010E94180D80E061E049E054E00E948E
:10630000080D89E061E04F2D5E2D0E94180D80E0A0
:106310006CED75E0A8010E94482F892B09F45FC03D
:1063200081E060EE75E04F2D5E2D0E94482F892B95
:1063300009F455C08091DB058093B5058091DC059B
:106340009091DD05A091DE05B091DF058093B80541
:106350009093B905A093BA05B093BB058091E00571
:106360009091E105A091E205B091E3058093BC0511
:106370009093BD05A093BE05B093BF0501C0A8953D
:10638000F999FDCF85E390E06091B5050E94F63D57
:1063900001C0A895F999FDCF4091B8055091B90574
:1063A0006091BA057091BB0586E390E00E94083EBB
:1063B00001C0A895F999FDCF4091BC055091BD054C
:1063C0006091BE057091BF058AE390E00E94083E8F
:1063D00006C08091DB05813009F043CFABCFE0965A
:1063E000E6E00C94173D1F93482F562F172F862F4A
:1063F000972F9C01D90124E630E0842F622F0E9460
:10640000923CE82F842F0E94923C492FF0E0E05DFF
:10641000FA4FE491ED93822F6AE00E94923C282F7C
:106420003F5F333051F7852F912F1F9108951F93B0
:106430005C9810E08FEF0E9487071F5F1031D1F743
:106440005C9A1F910895A8E0B0E0E9E2F2E30C94B1
:10645000F43C5C01E0910601FF27E7FDF095E55C67
:10646000FA4F749080E18CBD83E58CBD5C984B99AC
:1064700007C000E08FEF0E9487070F5F0830D1F759
:10648000D50116968C918E010F5F1F4FB8010E94A7
:10649000F3318B810E9487078A810E948707F5016B
:1064A00080858F5FB8010E94F3318B818F770E94C6
:1064B00087078A810E948707D5011A96ED90FC9084
:1064C0001B97ECE6F7E0EE0EFF1E90E1C92E97E277
:1064D000D92E86E0882E912C8C0E9D1EC701B60108
:1064E0000E949E3CE62FC701B6010E949E3C7C01A3
:1064F000F0E0E05DFA4FE491D801ED938D01C60123
:106500006AE070E00E949E3C6B010815190531F7A6
:106510008D818F770E9487078C810E9487078B81EE
:106520000E9487078A810E9487074B9B38C0809111
:10653000B505882311F40EEF05C0813011F007EF87
:1065400001C00FEB872D0E948707802F0E948707CD
:10655000F50180818E010F5F1F4FB8010E94F3315A
:106560008B810E9487078A810E948707D501129636
:106570008C91B8010E94F3318B818F770E9487073D
:106580008A810E948707F5018481B8010E94F33156
:106590008B818F770E9487078A810E9487075C9A88
:1065A00080E18CBD8CBD80E58CBD2896EDE00C941F
:1065B000103D682F88E048E455E00E94080D0895DA
:1065C000E82FF0E0EE0FFF1FE952FB4F4591549189
:1065D00080E061E00E94080D0895E82FF0E0EE0FE2
:1065E000FF1FE057FB4F4591549180E060E00E940F
:1065F000080D0895A4E0B0E0E0E0F3E30C94F73C6C
:10660000B82EA62E6A01FA0180817E010894E11C51
:10661000F11CB7010E94262B8E010E5F1F4F8B2DA0
:106620006A2DA8010E94180D8AE30E94AF0CF601A2
:106630008181B7010E94262BC8010E94B60C8AE313
:106640000E94AF0CF6018281B7010E94262BC8017F
:106650000E94B60C2496EAE00C94133DA3E0B0E04F
:10666000E4E3F3E30C94FA3CD82E7A018B01403436
:106670008EE7580785E0680780E0780738F088E003
:106680006D2D4FE355E00E94080D2EC0CB01BA01DD
:1066900020E13EE040E050E00E94D43C2983C80164
:1066A000B70120E13EE040E050E00E94D43C162FCC
:1066B000072FF82EE92E2CE330E040E050E00E9456
:1066C000D43C2A83612F702F8F2D9E2D2CE330E038
:1066D00040E050E00E94D43C6B8388E06D2DAE0119
:1066E0004F5F5F4F0E94FA322396E7E00C94163D0D
:1066F0008091BE04813049F44091B7045091B804B0
:106700006091B9047091BA041BC08731E1F48091A3
:10671000B3049091B404A091B504B091B6048F5F16
:106720009F4FAF4FBF4F19F4EDE0F5E015C040911A
:10673000AB045091AC046091AD047091AE0481E063
:106740000E942E330895883119F4EBE0F5E004C07F
:10675000893139F4E9E0F5E04591549188E061E050
:1067600004C088E061E048E455E00E94080D089507
:10677000AFE0B0E0EEEBF3E30C94F33C60901F016C
:106780007090210180902301A0902B01B0902C01EA
:1067900000912701109128010F5F1F4F9090250154
:1067A0008091290190912A0178E0C72ED12CCC0E3E
:1067B000DD1E8459984FB6010E94422B69E0E62EF7
:1067C000F12CEC0EFD1E80E060E0A7010E94180D88
:1067D0008FE20E94AF0C802FB6010E94262BC701CA
:1067E0000E94B60C8FE20E94AF0C892DB6010E9468
:1067F000262BC7010E94B60C80E20E94AF0C8E01CE
:106800000C5F1F4FAA0CBB1CAA0CBB1C8DE194E0B3
:10681000A80EB91EC801B5010E944B3DC8010E94D7
:10682000B60C80E20E94AF0CE0910601FF27E7FD65
:10683000F095E75CFB4FE4918E2F0E94AF0C8982AC
:106840007A826B8280E061E0AE014F5F5F4F0E9411
:10685000FA328091B505E82FF0E0EE0FFF1FE65DFC
:10686000FA4F4591549189E061E00E94080D80E261
:106870000E94AF0C5F9B02C08EE401C086E40E94C0
:10688000AF0C80E20E94AF0C8091090190910A0147
:10689000019711F480E501C080E20E94AF0C2F96B1
:1068A000EEE00C940F3DA0E1B0E0E9E5F4E30C94D8
:1068B000F93C0091A7050E94D70C002319F40E940F
:1068C000B83394C0013019F580E060E041E40E94E3
:1068D000230D6091DA027091DB028091DC029091CD
:1068E000DD028E010F5F1F4FA8010E948E2C0E94B7
:1068F000B60C80E061E04DE40E94230D6091DE0261
:106900007091DF028091E0029091E10224C0023098
:1069100041F580E060E047E40E94230D6091E202CF
:106920007091E3028091E4029091E5028E010F5F85
:106930001F4FA8010E948E2C0E94B60C80E061E0DF
:1069400044E40E94230D6091A3057091A4058091F9
:10695000A5059091A605A8010E948E2C0E94B60C58
:1069600045C0033009F580E060E043E955E00E944E
:10697000180D83E00E94E03204E0E0E0EE2EE1E05A
:10698000FE2E6E010894C11CD11CF70181917F017C
:10699000B6010E940E2BAC01802F61E00E94180D01
:1069A0000E5F003191F722C0043001F585E00E94AE
:1069B000ED328091090190910A01892B21F080919B
:1069C000B005882339F088E060E048E455E00E9493
:1069D000080D07C00E94CC04AB01BC0180E00E94FE
:1069E0002E3384E00E94E0320E9478336096E8E023
:1069F0000C94153DEF92FF920F93DF93CF93CDB799
:106A0000DEB760970FB6F894DEBF0FBECDBFA82FDC
:106A1000002309F461C07E010894E11CF11C88E0A8
:106A2000F70111928A95E9F729833A834B835C83B6
:106A30006D837E83AF83988780E2801BE82FFF27DA
:106A4000E7FDF09549815A816B817C81181684F0AD
:106A500019861A861B861C86882799278E1B9F0BF2
:106A600004C0440F551F661F771F8A95D2F728C0B0
:106A7000202F332727FD3095DB01CA01022E04C0E9
:106A8000880F991FAA1FBB1F0A94D2F789879A877C
:106A9000AB87BC8704C07695679557954795EA956F
:106AA000D2F78D819E81AF81B88504C0880F991F70
:106AB000AA1FBB1F2A95D2F7482B592B6A2B7B2B79
:106AC0004D875E876F87788B29853A854B855C85F6
:106AD0006D857E85AF8598898A2F60960FB6F8946C
:106AE000DEBF0FBECDBFCF91DF910F91FF90EF9032
:106AF0000895EF92FF920F93DF93CF93CDB7DEB758
:106B000060970FB6F894DEBF0FBECDBFA82F00234D
:106B100009F467C07E010894E11CF11C88E0F701CC
:106B200011928A95E9F729833A834B835C836D83BD
:106B30007E83AF83988780E2801B4D815E816F8169
:106B40007885E82FFF27E7FDF0951816B4F0DB01F4
:106B5000CA01BB0F880B982FDC018D879E87AF87FA
:106B6000B88B882799278E1B9F0B04C07595679556
:106B7000579547958A95D2F728C0202F332727FDB0
:106B80003095DB01CA01022E04C0B595A7959795F3
:106B900087950A94D2F78D879E87AF87B88B04C0FC
:106BA000440F551F661F771FEA95D2F789819A8196
:106BB000AB81BC8104C0B695A795979587952A951A
:106BC000D2F7482B592B6A2B7B2B49875A876B8727
:106BD0007C8729853A854B855C856D857E85AF856B
:106BE00098898A2F60960FB6F894DEBF0FBECDBF8E
:106BF000CF91DF910F91FF90EF900895AEE5B0E057
:106C0000E4E0F6E30C94EF3CA8E04E010894811C0C
:106C1000911CF4016A2E11926A94E9F729833A8350
:106C20004B835C836D837E838F839887CE01099627
:106C3000FC011192AA95E9F7A986BA86CB86DC8673
:106C4000ED86FE860F87188B29843A844B845C84FA
:106C5000ED84FE840F85188969807A808B809C8002
:106C60006DA67EA68FA698AA6D807E808F80988460
:106C7000E114F1040105110509F0B3C362147304B2
:106C80008404950408F03DC100E0201600E03006C1
:106C900001E0400600E0500688F41FEF21163104A1
:106CA0004104510439F030F048E0E42EF12C012D7C
:106CB000112D18C0EE24FF24870114C020E02216F5
:106CC00020E0320620E0420621E0520630F038E1B2
:106CD000E32EF12C012D112D05C020E1E22EF12C27
:106CE000012D112DD201C1010E2C04C0B695A7951E
:106CF000979587950A94D2F787599E4FDC012C917E
:106D000080E290E0A0E0B0E08E199F09A00BB10BEB
:106D10007C018D01E21AF10801091109E114F10465
:106D200001051105A1F10E2C04C0220C331C441CDA
:106D3000551C0A94D2F7A40193010E2C04C0220F13
:106D4000331F441F551F0A94D2F780E290E08E193A
:106D50009F096DA47EA48FA498A804C096948794DC
:106D6000779467948A95D2F7622A732A842A952A9F
:106D7000ADA4BEA4CFA4D8A804C0AA0CBB1CCC1C34
:106D8000DD1CEA94D2F7ADA6BEA6CFA6D8AA6201B2
:106D9000EE24FF24CDAADEAAEFAAF8AE920181016B
:106DA0002070307009AF1AAF2BAF3CAFC401B301F4
:106DB000A70196010E94B23C7B018C01C401B30182
:106DC0002DA93EA94FA958AD0E94B23CC901DA01D4
:106DD0003C014D01C401B30129AD3AAD4BAD5CADF1
:106DE0000E94733C9B01AC018701FF24EE24ADA4FB
:106DF000BEA4CFA4D8A8C601AA27BB275701680103
:106E0000A82AB92ACA2ADB2AA216B306C406D506BE
:106E1000E0F408946108710881089108A20CB31C81
:106E2000C41CD51CA214B304C404D50470F0A2166B
:106E3000B306C406D50648F40894610871088108B1
:106E40009108A20CB31CC41CD51CA21AB30AC40A14
:106E5000D50AC601B5012DA93EA94FA958AD0E947A
:106E6000B23C7B018C01C601B5012DA93EA94FA9F9
:106E700058AD0E94B23CC901DA015C016D01C60146
:106E8000B50129AD3AAD4BAD5CAD0E94733C9B01A1
:106E9000AC018701FF24EE248DA59EA5AFA5B8A95E
:106EA000A070B070E82AF92A0A2B1B2BE216F30611
:106EB00004071507C0F40894A108B108C108D10857
:106EC000E20CF31C041D151DE214F3040405150562
:106ED00050F0E216F3060407150728F40894A108F9
:106EE000B108C108D108D301992788278601750107
:106EF000E82AF92A0A2B1B2BE9AAFAAA0BAB1CAB2E
:106F0000CFC4211431044104510471F461E070E0F4
:106F100080E090E020E030E040E050E00E94B23CB1
:106F2000C901DA011C012D0100E0201600E0300645
:106F300001E0400600E0500688F41FEF21163104FE
:106F40004104510431F028F048E050E060E070E086
:106F500017C040E050E060E070E012C020E0221670
:106F600020E0320620E0420621E0520628F048E107
:106F700050E060E070E004C040E150E060E070E0AC
:106F8000D201C101042E04C0B695A79597958795A7
:106F90000A94D2F787599E4FDC012C91E0E2EE2E45
:106FA000F12C012D112DD801C701841B950BA60BC7
:106FB000B70B821B9109A109B1090097A105B10581
:106FC00061F464015301A218B308C408D50831E084
:106FD000632E712C812C912C1EC16F968FAF6F97F1
:106FE000082E04C0220C331C441C551C0A94D2F7F2
:106FF000EE2DE81B640153010E2E04C0D694C794F5
:10700000B794A7940A94D2F7A40193016F960FAC9A
:107010006F9704C0220F331F441F551F0A94D2F7E5
:107020006DA47EA48FA498A80E2E04C09694879475
:10703000779467940A94D2F784017301E22AF32AC1
:10704000042B152BE9A6FAA60BA71CA7320188244E
:107050009924920181012070307021960CAF1DAFF0
:107060002EAF3FAF2197C601B501A40193010E9445
:10707000B23C7B018C01C601B501A40193010E94C1
:10708000B23CC901DA0125968CAF9DAFAEAFBFAF60
:107090002597BC01CD0121962CAD3DAD4EAD5FAD28
:1070A00021970E94733C9B01AC018701FF24EE24D1
:1070B000A9A4BAA4CBA4DCA4C601AA27BB275C015F
:1070C0006D01AE28BF28C02AD12AA216B306C40675
:1070D000D50660F525966CAD7DAD8EAD9FAD25973F
:1070E000615070408040904025966CAF7DAF8EAF70
:1070F0009FAF2597A20CB31CC41CD51CA214B304CB
:10710000C404D50498F0A216B306C406D50670F4DC
:10711000615070408040904025966CAF7DAF8EAF3F
:107120009FAF2597A20CB31CC41CD51CA21AB30A8E
:10713000C40AD50AC601B501A40193010E94B23C5C
:107140007B018C01C601B501A40193010E94B23CF0
:10715000C901DA013C014D01C401B30121962CADF6
:107160003DAD4EAD5FAD21970E94733C9B01AC01DC
:107170008701FF24EE2489A59AA5ABA5BCA5A07024
:10718000B07057016801A82AB92ACA2ADB2AA216B8
:10719000B306C406D506E0F40894610871088108B6
:1071A0009108A20CB31CC41CD51CA214B304C404C3
:1071B000D50470F0A216B306C406D50648F40894A8
:1071C0006108710881089108A20CB31CC41CD51C6D
:1071D0008DA59EA5AFA5B8A96F960FAC6F9704C0FB
:1071E000880F991FAA1FBB1F0A94D2F78DA79EA7CD
:1071F000AFA7B8ABA21AB30AC40AD50A2596ECAC5D
:10720000FDAC0EAD1FAD2597D70199278827682AB9
:10721000792A8A2A9B2A82012227332729960CAFB2
:107220001DAF2EAF3FAF2997A20191014070507062
:107230002D962CAF3DAF4EAF5FAF2D97C601B50178
:1072400029962CAD3DAD4EAD5FAD29970E94B23C65
:107250007B018C01C601B50129962CAD3DAD4EAD2B
:107260005FAD29970E94B23CC901DA0161968CAFEB
:107270009DAFAEAFBFAF6197BC01CD012D962CADD8
:107280003DAD4EAD5FAD2D970E94733C9B01AC01AF
:107290008701FF24EE24ADA4BEA4CFA4D8A8C601C4
:1072A000AA27BB2757016801A82AB92ACA2ADB2ABC
:1072B000A216B306C406D50660F561966CAD7DAD29
:1072C0008EAD9FAD61976150704080409040619657
:1072D0006CAF7DAF8EAF9FAF6197A20CB31CC41C87
:1072E000D51CA214B304C404D50498F0A216B306A6
:1072F000C406D50670F4615070408040904061969D
:107300006CAF7DAF8EAF9FAF6197A20CB31CC41C56
:10731000D51CA21AB30AC40AD50AC601B50129961A
:107320002CAD3DAD4EAD5FAD29970E94B23C7B01C7
:107330008C01C601B50129962CAD3DAD4EAD5FADBA
:1073400029970E94B23CC901DA015C016D01C601B6
:10735000B5012D962CAD3DAD4EAD5FAD2D970E9484
:10736000733C9B01AC018701FF24EE248DA59EA5F3
:10737000AFA5B8A9A070B070E82AF92A0A2B1B2B78
:10738000E216F30604071507C0F40894A108B10833
:10739000C108D108E20CF31C041D151DE214F3040E
:1073A0000405150550F0E216F3060407150728F446
:1073B0000894A108B108C108D1086196ECACFDACF5
:1073C0000EAD1FAD6197D7019927882796018501DA
:1073D000082B192B2A2B3B2B09AB1AAB2BAB3CAB45
:1073E00062C26E147F048006910608F451C220E048
:1073F000E21620E0F20621E0020720E0120788F4FE
:107400003FEFE316F1040105110531F028F048E0E3
:1074100050E060E070E017C040E050E060E070E0F5
:1074200012C040E0E41640E0F40640E0040741E00A
:10743000140728F048E150E060E070E004C040E14B
:1074400050E060E070E0D801C701042E04C0B6959A
:10745000A795979587950A94D2F787599E4FDC0197
:107460002C9130E2A32EB12CC12CD12CD601C50118
:10747000841B950BA60BB70B821B9109A109B109BF
:107480000097A105B10589F4E614F704080519056C
:1074900008F4F2C16DA47EA48FA498A862147304AA
:1074A0008404950408F0E8C1F3C16E968FAF6E971F
:1074B000082E04C0EE0CFF1C001F111F0A94D2F707
:1074C0006A2D681BD201C101062E04C0B695A7958E
:1074D000979587950A94D2F75C016D01AE28BF2875
:1074E000C02AD12AADA2BEA2CFA2D8A67201610144
:1074F0006E960FAC6E9704C0CC0CDD1CEE1CFF1C0E
:107500000A94D2F7C9A2DAA2EBA2FCA26401530149
:10751000062E04C0D694C794B794A7940A94D2F7C1
:10752000D401C3016E960FAC6E9704C0880F991FEB
:10753000AA1FBB1F0A94D2F7EDA4FEA40FA518A999
:1075400004C016950795F794E7946A95D2F737012A
:107550004801682A792A8A2A9B2A6D8E7E8E8F8E10
:1075600098A2EDA0FEA00FA118A5380188249924A7
:10757000980187012070307065960CAF1DAF2EAF5B
:107580003FAF6597C601B501A40193010E94B23CCB
:107590007B018C01C601B501A40193010E94B23C9C
:1075A000C901DA011C012D01C201B10165962CADA2
:1075B0003DAD4EAD5FAD65970E94733C9B01AC0144
:1075C0008701FF24EE24AD8CBE8CCF8CD8A0C601E1
:1075D000AA27BB2757016801A82AB92ACA2ADB2A89
:1075E000A216B306C406D50600F508942108310892
:1075F00041085108EDA0FEA00FA118A5AE0CBF1CBC
:10760000C01ED11EAE14BF04C006D10670F0A21673
:10761000B306C406D50648F4089421083108410889
:107620005108AE0CBF1CC01ED11EA21AB30AC40A58
:10763000D50AC601B501A40193010E94B23C7B01A9
:107640008C01C601B501A40193010E94B23CC9019D
:10765000DA013C014D01C401B30165962CAD3DAD8D
:107660004EAD5FAD65970E94733C9B01AC018701F5
:10767000FF24EE248D8D9E8DAF8DB8A1A070B070CB
:1076800057016801A82AB92ACA2ADB2AA216B3061A
:10769000C406D50600F508946108710881089108B0
:1076A0006DA17EA18FA198A5A60EB71EC81ED91EDA
:1076B000A616B706C806D90670F0A216B306C40609
:1076C000D50648F408946108710881089108A60E4F
:1076D000B71EC81ED91ED601C501821B930BA40B71
:1076E000B50B898F9A8FAB8FBC8FD10199278827D3
:1076F00064015301A82AB92ACA2ADB2AA9AABAAA6C
:10770000CBAADCAA860175012FEF3FEF40E050E0E5
:10771000E222F32204231523A601662777276D961C
:107720004CAF5DAF6EAF7FAF6D97A9A0BAA0CBA0F5
:10773000DCA06FEF7FEF80E090E0A622B722C822A6
:10774000D92289A19AA1ABA1BCA11D014424552431
:10775000C801B701A60195010E94733C69966CAF00
:107760007DAF8EAF9FAF6997C801B701A2019101AC
:107770000E94733C3B014C016D966CAD7DAD8EADAE
:107780009FAD6D97A60195010E94733C7B018C0112
:107790006D966CAD7DAD8EAD9FAD6D97A2019101E3
:1077A0000E94733C5B016C01A8019701260D371DF7
:1077B000481D591D69966CAC7DAC8EAC9FAC699729
:1077C000C401AA27BB27280F391F4A1F5B1F2E158C
:1077D0003F054007510748F4E12CF12C61E0062FEA
:1077E000112DAE0CBF1CC01ED11ECA01AA27BB277B
:1077F000BC01CD016A0D7B1D8C1D9D1D698C7A8C91
:107800008B8C9C8C661677068806990640F1661567
:1078100077058805990509F043C0D901992788277C
:1078200069962CAD3DAD4EAD5FAD6997407050701F
:10783000820F931FA41FB51F2DA53EA54FA558A9C4
:107840006E960FAC6E9704C0220F331F441F551F56
:107850000A94D2F7281739074A075B0708F509A9E0
:107860001AA92BA93CA9015010402040304009AB77
:107870001AAB2BAB3CAB14C066247724430121E048
:1078800030E040E050E029AB3AAB4BAB5CAB0BC017
:1078900066247724430119AA1AAA1BAA1CAA03C0AA
:1078A000662477244301FE01719688E0DF011D9272
:1078B0008A95E9F7A9A8BAA8CBA8DCA8A98ABA8AA8
:1078C000CB8ADC8A6D8A7E8A8F8A988E29A93A892A
:1078D0004B895C89662D7E898F89988DC25ADF4FCE
:1078E000E2E10C940B3D629FD001739FF001829FF7
:1078F000E00DF11D649FE00DF11D929FF00D839F3F
:10790000F00D749FF00D659FF00D9927729FB00DDB
:10791000E11DF91F639FB00DE11DF91FBD01CF01EE
:1079200011240895991B79E004C0991F961708F057
:10793000961B881F7A95C9F780950895AA1BBB1BD3
:1079400051E107C0AA1FBB1FA617B70710F0A61B5F
:10795000B70B881F991F5A95A9F780959095BC0180
:10796000CD010895A1E21A2EAA1BBB1BFD010DC07B
:10797000AA1FBB1FEE1FFF1FA217B307E407F507DF
:1079800020F0A21BB30BE40BF50B661F771F881FBB
:10799000991F1A9469F760957095809590959B0151
:1079A000AC01BD01CF01089597FB092E05260ED02D
:1079B00057FD04D0D7DF0AD0001C38F4509540950D
:1079C000309521953F4F4F4F5F4F0895F6F79095B3
:1079D0008095709561957F4F8F4F9F4F08952F929F
:1079E0003F924F925F926F927F928F929F92AF924F
:1079F000BF92CF92DF92EF92FF920F931F93CF939C
:107A0000DF93CDB7DEB7CA1BDB0B0FB6F894DEBF32
:107A10000FBECDBF09942A88398848885F846E8458
:107A20007D848C849B84AA84B984C884DF80EE80A2
:107A3000FD800C811B81AA81B981CE0FD11D0FB6AB
:107A4000F894DEBF0FBECDBFED010895911106C0C1
:107A500080538A5010F0865C06C0089599278827C5
:107A6000089585FDFBCF80629111F8CF81568A5130
:107A7000E0F708959111089581568A5108F48052D3
:107A800085580895FB01DC018D9105908019011046
:107A9000D9F3990B0895FB01DC0105900D920020AC
:107AA000E1F70895FC0105900020E9F78095909595
:107AB0008E0F9F1F0895FB01DC014150504030F0B4
:107AC0008D910590801919F40020B9F7881B990B46
:107AD0000895FB0155915523A9F0BF01DC014D919B
:107AE00045174111E1F759F4CD010590002049F007
:107AF0004D9140154111C9F3FB014111EFCF81E0D8
:107B000090E001970895DC0101C06D934150504011
:107B1000E0F70895FC018191861721F08823D9F7B9
:107B2000992708953197CF010895FB01DC018D91CC
:107B3000019080190110D9F3990B0895FB01DC0124
:107B400001900D920020E1F70895FB01DC01415006
:107B5000504030F08D910190801919F40020B9F750
:107B6000881B990B0895FB01DC014150504048F0FF
:107B700001900D920020C9F701C01D924150504064
:107B8000E0F70895DC01CB01FC01F999FECF06C0B6
:107B9000F2BDE1BDF89A319600B40D9241505040CB
:107BA000B8F70895F999FECF92BD81BDF89A99274B
:107BB00080B50895A6E1B0E044E050E00C94C43DE7
:107BC000A8E1B0E042E050E00C94C43DDC01A40F19
:107BD000B51F4150504048F0CB01840F951F2E91A6
:107BE0000E94F73D41505040D0F70895262FF99953
:107BF000FECF92BD81BDF89A019700B4021639F00C
:107C00001FBA20BD0FB6F894FA9AF99A0FBE0895DC
:107C10000396272F0E94F73D0E94F63D252F0E94D4
:107C2000F73D242F0C94F73DDC01CB0103C02D91CF
:107C30000E941F3E41505040D0F70895262FF999D9
:107C4000FECF1FBA92BD81BD20BD0FB6F894FA9A3F
:107C5000F99A0FBE01960895242F0E941F3E252FEA
:107C60000E941F3E0C94343E0E941E3E272F0C940F
:067C70001F3EF894FFCF57
:107C760002000000000002C0100100000000000920
:107C860000010000004600000000000000010000A6
:107C9600000000090001000000460000000000008E
:107CA6000000000000000001000000460000000087
:107CB600000000000000000900010000004600006E
:107CC6000000000000907E000015CD5B07E5559A88
:107CD60015B53B121F3313490500010202030303C6
:107CE6000304040404040404040505050505050548
:107CF6000505050505050505050606060606060627
:107D0600060606060606060606060606060606060D
:107D160006060606060606060607070707070707F6
:107D260007070707070707070707070707070707DD
:107D360007070707070707070707070707070707CD
:107D460007070707070707070707070707070707BD
:107D560007070707070707070708080808080808A6
:107D6600080808080808080808080808080808088D
:107D7600080808080808080808080808080808087D
:107D8600080808080808080808080808080808086D
:107D9600080808080808080808080808080808085D
:107DA600080808080808080808080808080808084D
:107DB600080808080808080808080808080808083D
:107DC600080808080808080808080808080808082D
:0A7DD600080808080808080808005B
:00000001FF
